:1000000002630502594EAB07AA06900000C3E582C1
:100010009BEA6480F8E583648098500612776DA3AC
:1000200080EB22026EE6780AE6FF22026748900E15
:100030005E7401F0A3740DF0A3742AF0900E5D7449
:100040000AF0220258A1E709F608DFFA8046E7091C
:10005000F208DFFA803E88828C83E709F0A3DFFA9A
:100060008032E309F608DFFA8078E309F208DFFA64
:10007000807088828C83E309F0A3DFFA8064898230
:100080008A83E0A3F608DFFA805889828A83E0A396
:10009000F208DFFA804C80D280FA80C680D4806972
:1000A00080F28033801080A680EA809A80A880DA6F
:1000B00080E280CA803389828A83ECFAE493A3C801
:1000C000C582C8CCC583CCF0A3C8C582C8CCC583C3
:1000D000CCDFE9DEE7800D89828A83E493A3F6080A
:1000E000DFF9ECFAA9F0EDFB2289828A83ECFAE0D1
:1000F000A3C8C582C8CCC583CCF0A3C8C582C8CC70
:10010000C583CCDFEADEE880DB89828A83E493A3BF
:10011000F208DFF980CC88F0EF60010E4E60C388F2
:10012000F0ED2402B4040050B9F582EB2402B404CB
:100130000050AF232345822390009673C2D530F739
:1001400007B2D563F0FF05F030E70CB2D5F40484B4
:1001500063F0FF05F080018430D502F40422BB0176
:100160000689828A83E0225002E722BBFE02E32254
:1001700089828A83E49322BB010989828A83F8E019
:1001800028F022500327F722BBFE05F8E328F322CC
:100190008A838982F8E4932822BB010689828A83B4
:1001A000F0225002F722BBFE01F322EF8DF0A4A84B
:1001B000F0CF8CF0A428CE8DF0A42EFE22C2D5EC78
:1001C00030E709B2D5E4C39DFDE49CFCEE30E715B1
:1001D000B2D5E4C39FFFE49EFE12060EC3E49DFD6C
:1001E000E49CFC800312060E30D507C3E49FFFE4B5
:1001F0009EFE22C5F0F8A3E028F0C5F0F8E58215D0
:100200008270021583E038F022A3F8E0C5F025F0F3
:10021000F0E582158270021583E0C838F0E822BB51
:10022000010A89828A83E0F5F0A3E022500687F074
:1002300009E71922BBFE07E3F5F009E319228982D9
:100240008A83E493F5F074019322BB010A89828AC0
:1002500083F0E5F0A3F0225006F709A7F01922BBBE
:10026000FE06F3E5F009F31922E88FF0A4CC8BF039
:10027000A42CFCE98EF0A42CFC8AF0EDA42CFCEA62
:100280008EF0A4CDA8F08BF0A42DCC3825F0FDE99C
:100290008FF0A42CCD35F0FCEB8EF0A4FEA9F0EB92
:1002A0008FF0A4CFC5F02ECD39FEE43CFCEAA42D9E
:1002B000CE35F0FDE43CFC2275F008758200EF2F8E
:1002C000FFEE33FECD33CDCC33CCC58233C5829B1C
:1002D000ED9AEC99E58298400CF582EE9BFEED9A42
:1002E000FDEC99FC0FD5F0D6E4CEFBE4CDFAE4CCDE
:1002F000F9A88222B800C1B90059BA002DEC8BF0E0
:1003000084CFCECDFCE5F0CBF97818EF2FFFEE339C
:10031000FEED33FDEC33FCEB33FB10D703994004C7
:10032000EB99FB0FD8E5E4F9FA227818EF2FFFEEEE
:1003300033FEED33FDEC33FCC933C910D7059BE91F
:100340009A4007EC9BFCE99AF90FD8E0E4C9FAE47B
:10035000CCFB2275F010EF2FFFEE33FEED33FDCC1A
:1003600033CCC833C810D7079BEC9AE899400AED04
:100370009BFDEC9AFCE899F80FD5F0DAE4CDFBE4AC
:10038000CCFAE4C8F922EB9FF5F0EA9E42F0E99D31
:1003900042F0EC6480C864809845F022EB9FF5F051
:1003A000EA9E42F0E99D42F0E89C45F022E8600FA9
:1003B000ECC313FCED13FDEE13FEEF13FFD8F12297
:1003C000E8600FEFC333FFEE33FEED33FDEC33FC9B
:1003D000D8F122ECF0A3EDF0A3EEF0A3EFF022D0E1
:1003E00083D082F8E4937012740193700DA3A393E9
:1003F000F8740193F5828883E4737402936860EF64
:10040000A3A3A380DF8A838982E473EC8EF0A4CC5B
:10041000C5F0CCCDF8EFA4CEC5F02DFDE43CFCE852
:10042000A42EC8C5F03DFDE43CFCEFA4FFE5F02898
:10043000FEE43DFDE43CFC22E3F5F009E208B5F002
:100440006BDFF58067E3F5F009E608B5F05EDFF5F0
:10045000805A87F009E608B5F052DFF6804E87F043
:1004600009E208B5F046DFF6804288828C8387F087
:1004700009E0A3B5F036DFF6803288828C8387F0FE
:1004800009E493A3B5F025DFF5802188828C83E30E
:10049000F5F009E0A3B5F014DFF5801088828C83B5
:1004A000E3F5F009E493A3B5F002DFF402056780F9
:1004B0008780E9809080D4803E8015806E807E8029
:1004C0009D80B7808D80A380518074803C0205732D
:1004D00089828A83ECFAE493F5F0A3C8C582C8CC7C
:1004E000C583CCE493A3C8C582C8CCC583CCB5F082
:1004F00076DFE3DEE1807089828A83E493F5F0A3FE
:10050000E208B5F062DFF4805E89828A83E0F5F06C
:10051000A3E608B5F051DFF5804D89828A83E0F5C6
:10052000F0A3E208B5F040DFF5803C89828A83E4DD
:1005300093F5F0A3E608B5F02EDFF4802A80028060
:100540005789828A83ECFAE493F5F0A3C8C582C880
:10055000CCC583CCE0A3C8C582C8CCC583CCB5F0DC
:1005600006DFE4DEE280007FFFB5F0020F224002EA
:100570007F012289828A83ECFAE0F5F0A3C8C58264
:10058000C8CCC583CCE0A3C8C582C8CCC583CCB5D4
:10059000F0D5DFE5DEE380CF89828A83ECFAE0F5EF
:1005A000F0A3C8C582C8CCC583CCE493A3C8C582D8
:1005B000C8CCC583CCB5F0AFDFE4DEE280A988F01B
:1005C000EF60010E4E60ABED2402B404005098F5CC
:1005D00082EB2402B40400508E232345822390042E
:1005E000AF73EF4E6012EF60010EEDBB010B89821D
:1005F0008A83F0A3DFFCDEFA2289F05007F709DFD7
:10060000FCA9F022BBFEFCF309DFFCA9F022BC0030
:100610000BBE0029EF8DF084FFADF022E4CCF8751D
:10062000F008EF2FFFEE33FEEC33FCEE9DEC98402C
:1006300005FCEE9DFE0FD5F0E9E4CEFD22EDF8F5C8
:10064000F0EE8420D21CFEADF075F008EF2FFFED28
:1006500033FD4007985006D5F0F222C398FD0FD520
:10066000F0EA22E4FFFEFDFC900C651203D3900C2F
:1006700065E0F8A3E0F9A3E0FAA3E0FB900E20E028
:10068000FFE4FCFDFEEB2FFFEE3AFEED39FDEC380A
:10069000FC900C651203D3900C65E0F8A3E0F9A37D
:1006A000E0FAA3E0FBC000900E21E0FFE4FCFDFEB9
:1006B00078081203C0D000EB2FFFEA3EFEE93DFDB3
:1006C000E83CFC900C651203D3900C65E0F8A3E0C5
:1006D000F9A3E0FAA3E0FBC000900E22E0FFE4FCE7
:1006E000FDFE78101203C0D000EB2FFFEA3EFEE9BA
:1006F0003DFDE83CFC900C651203D3900E1FE024F6
:10070000FE70030207B024FE70030207DB24FC70B6
:10071000030208AA24F870030209041470030209F2
:100720008424F17003020A69241F6003020B96906F
:100730000C65E0FCA3E0FDA3E0FEA3E0FF900C72DB
:100740001203D37F161217E7900C64748BF01278A3
:1007500073900C64E0241BF0E0FF12481D900C69BC
:10076000EFF0900C767401F0A3740CF0A37463F0B6
:100770007B017A0C7962E4FFFE12344D900C62E04A
:10078000540FC3940E400A900C64E06480946C4053
:10079000C0127829900C62E0FE540F900D6EF0EEBE
:1007A000C4540FA3F0900C63E0900D70F0020B9E08
:1007B000900C65E0FCA3E0FDA3E0FEA3E0FF900C3D
:1007C000721203D37F161217E7122BB2AD07AC06D5
:1007D000EF900D6EF0EEA3F0020B9E90000CE00483
:1007E000F0900B53E004F090000CE0FBD394354004
:1007F0000A7435F0E4900D6E020B9B900C65E0FCE2
:10080000A3E0FDA3E0FEA3E0FF75F004EBA4240940
:10081000F582E5F03400F5831203D3900E23E0FF58
:1008200074E02BF582E43400F583EFF0900E24E0C1
:10083000900B54F0900C65E0FCA3E0FDA3E0FEA358
:10084000E0FF900008E0F8A3E0F9A3E0FAA3E0FBE2
:10085000C312039C5014900C65E0FCA3E0FDA3E0E0
:10086000FEA3E0FF9000081203D3900C65E0FCA308
:10087000E0FDA3E0FEA3E0FF900B4FE0F8A3E0F95A
:10088000A3E0FAA3E0FBD312039C4014900C65E0B4
:10089000FCA3E0FDA3E0FEA3E0FF900B4F1203D307
:1008A000900D6E74FCF0A302097E90000C7401F0B0
:1008B000900B53F0900C65E0FCA3E0FDA3E0FEA3D9
:1008C000E0FF90000D1203D3900E23E09000E1F0C2
:1008D000900C65E0FCA3E0FDA3E0FEA3E0FF900028
:1008E000081203D3900C65E0FCA3E0FDA3E0FEA397
:1008F000E0FF900B4F1203D3900D6E74FEF0A30433
:10090000F0020B9E900E20E0FF7E00900B48EEF070
:10091000A3EFF0FD900E21E0FFED900B48CFF0A388
:10092000EFF0900E22E0FF900B18EEF0A3EFF0FD39
:10093000900E23E0FFED900B18CFF0A3EFF0900E98
:1009400024E0FF900B3AEEF0A3EFF0FD900E25E0CF
:10095000FFED900B3ACFF0A3EFF0900D6E74FEF028
:10096000C3900B19E09432900B18E09400500CE403
:10097000F0A37432F0900D6E74FFF0900D6F74FF61
:10098000F0020B9EE4FFFEFDFC900C691203D37491
:10099000FFFFFEFDFC900C6D1203D3900D6E74FEF4
:1009A000F0A304F0900B54E0900D70F0900B48E031
:1009B000FCA3E0900D71F0ECA3F0900B18E0FCA309
:1009C000E0900D73F0ECA3F0900B3AE0FCA3E09004
:1009D0000D75F0ECA3F0900B4FE0FCA3E0FDA3E05D
:1009E000FEA3E0FF900D77EFF0900B4FA3A3A3E0E1
:1009F00078081203AD900D78EFF0900B4FE0FCA358
:100A0000E0FDA3E0FEA3E0FF78101203AD900D79A6
:100A1000EFF0900008E0FCA3E0FDA3E0FEA3E0FF00
:100A2000900D7AEFF0900008A3A3A3E078081203DA
:100A3000AD900D7BEFF0900008E0FCA3E0FDA3E09B
:100A4000FEA3E0FF78101203AD900D7CEFF0900B49
:100A500053E0900D7DF09000E1E0900D7EF090006D
:100A60000CE0900D7FF0020B9E900E24E0FE900EA5
:100A700023E0FDEDFF900C69EEF0A3EFF07F07128D
:100A800073C9900C6BEFF07F081273C9900C6CEF78
:100A9000F0E4FD7F0712757AE4FD7F0812757A9005
:100AA0000C65E0FCA3E0FDA3E0FEA3E0FF900C7268
:100AB0001203D37F161217E7900D6C7442F0A374E3
:100AC00040F0900E73E0FBA3E0FAA3E02401F9E408
:100AD0003AFA12015E900E72F0A37401F0A3740D45
:100AE000F0A3746CF0900D6E74FEF0A304F0127518
:100AF00020900C69E0FEA3E0FFD394E8EE9403405D
:100B00001BEF2420FFE43EFEEF7806CEC313CE1386
:100B1000D8F9FF7C007D301201AB801A900C69E09F
:100B2000FEA3E0FF7C007D301201ABEF7806CEC360
:100B300013CE13D8F9FF900B3FEEF0A3EFF0E49043
:100B40000B42F012768C12797B7F011274627F8FD8
:100B50001276B07F9E1276B07D0A7C007F807E0088
:100B6000126D22E4900B59F0A3F01275F3EF6006BA
:100B7000120026EF60D8E4FF127462900C6BE0FD67
:100B80007F0712757A900C6CE0FD7F0812757A90E1
:100B90000B477401F022900D6E74FFF0A3F0900DDE
:100BA0006C7442F0A37440F0900E73E0FBA3E0FA83
:100BB000A3E02401F9E43AFA12015E900E72F0A368
:100BC0007401F0A3740DF0A3746CF012752022E48C
:100BD000900C5CF0900C5FF0A374C8F0A37401F06B
:100BE00053D9BF1278F3D2AF1272D81278847BFF38
:100BF0007A68797812108B7F5E7EC67D0D7C0090BE
:100C0000000D1203D39000E174D8F07F527EC87DAE
:100C10000D7C009000111203D39000E274D8F07F95
:100C2000467ECA7D0D7C009000151203D39000E330
:100C300074D8F07F3A7ECC7D0D7C009000191203B1
:100C4000D39000E474D8F07F2E7ECE7D0D7C009092
:100C5000001D1203D39000E574D8F07F227ED07D72
:100C60000D7C009000211203D39000E674D8F07F31
:100C7000167ED27D0D7C009000251203D39000E7F4
:100C800074D8F07F0A7ED47D0D7C00900029120379
:100C9000D39000E874D8F07FFE7ED57D0D7C009067
:100CA000002D1203D39000E974D8F07FF27ED77D37
:100CB0000D7C009000311203D39000EA74D8F07FCD
:100CC000E67ED97D0D7C009000351203D39000EBB9
:100CD00074D8F07FDA7EDB7D0D7C00900039120342
:100CE000D39000EC74D8F07FCE7EDD7D0D7C00903B
:100CF000003D1203D39000ED74D8F07FC27EDF7DFB
:100D00000D7C009000411203D39000EE74D8F07F68
:100D1000B67EE17D0D7C009000451203D39000EF7C
:100D200074D8F07FAA7EE37D0D7C00900049120309
:100D3000D39000F074D8F07F9E7EE57D0D7C00900E
:100D4000004D1203D39000F174D8F07F927EE77DBE
:100D50000D7C009000511203D39000F274D8F07F04
:100D6000867EE97D0D7C009000551203D39000F340
:100D700074D8F07F7A7EEB7D0D7C009000591203D1
:100D8000D39000F474D8F07F6E7EED7D0D7C0090E2
:100D9000005D1203D39000F574D8F07F627EEF7D82
:100DA0000D7C009000611203D39000F674D8F07FA0
:100DB000567EF17D0D7C009000651203D39000F704
:100DC00074D8F07F4A7EF37D0D7C00900069120399
:100DD000D39000F874D8F07F3E7EF57D0D7C0090B6
:100DE000006D1203D39000F974D8F07F327EF77D46
:100DF0000D7C009000711203D39000FA74D8F07F3C
:100E0000267EF97D0D7C009000751203D39000FBC7
:100E100074D8F07F1A7EFB7D0D7C00900079120360
:100E2000D39000FC74D8F07F0E7EFD7D0D7C009089
:100E3000007D1203D39000FD74D8F07F027EFF7D09
:100E40000D7C009000811203D39000FE74D8F07FD7
:100E50005C7E797D0C7C009000851203D39000FFAE
:100E600074D8F07FEA7E027D0E7C00900089120328
:100E7000D390010074D8F07FDE7E047D0E7C00905C
:100E8000008D1203D390010174D8F07FD27E067DCD
:100E90000E7C009000911203D390010274D8F07F71
:100EA000C67E087D0E7C009000951203D39001034E
:100EB00074D8F07FBA7E0A7D0E7C009000991203F0
:100EC000D390010474D8F07FAE7E0C7D0E7C009030
:100ED000009D1203D390010574D8F07FA27E0E7D91
:100EE0000E7C009000A11203D390010674D8F07F0D
:100EF000967E107D0E7C009000A51203D390010712
:100F000074D8F07F8A7E127D0E7C009000A91203B7
:100F1000D390010874D8F07F7E7E147D0E7C009003
:100F200000AD1203D390010974D8F07F727E167D54
:100F30000E7C009000B11203D390010A74D8F07FA8
:100F4000667E187D0E7C009000B51203D390010BD5
:100F500074D8F07F5A7E1A7D0E7C009000B912037F
:100F6000D390010C74D8F07F4E7E1C7D0E7C0090D7
:100F700000BD1203D390010D74D8F07F427E1E7D18
:100F80000E7C009000C11203D390010E74D8F07F44
:100F9000367E207D0E7C009000C51203D390010F99
:100FA00074D8F07F2A7E227D0E7C009000C9120347
:100FB000D390011074D8F07F1E7E247D0E7C0090AB
:100FC00000CD1203D390011174D8F07F127E267DDC
:100FD0000E7C009000D11203D390011274D8F090CF
:100FE000000C7432F0A3E0FCA3E0FDA3E0FEA3E05C
:100FF000FF121DB9900C5DEEF0A3EFF04E60177F6D
:10100000E87E031276F5900C5DA3E0FF125EF97F97
:10101000E87E031276F57BFF7A687994900C5DE0A8
:10102000FFA3E0900CD3CFF0A3EFF012108B127857
:10103000FD900C5FE07002A3E06010900C60E02473
:10104000FFF0900C5FE034FFF0803B900C5DE070AF
:1010500002A3E07F0060027F0474C07E5DA80708E1
:101060008005C333CE33CED8F9900C60F0EE900CEF
:101070005FF0900C61E06006E4F0C2A28008900C82
:10108000617401F0D2A212470F80A6900CD0EBF051
:10109000A3EAF0A3E9F0E4900CFBF0A3F0A3F0A323
:1010A000F0A3F0A3F0A3F0A3F0900D07F0A3F0A33A
:1010B000F0A3F0A3F0900D1304F0A3740CF0A3744C
:1010C000D3F0900CD0E0FBA3E0FAA3E0F912015EAC
:1010D00070030214C41203DF147E0A111B25141AB4
:1010E000301440311440321440331440341440352D
:1010F00014403614403714403814403911724411EA
:101100007255116A58117263117264113D6811723F
:101110006C11727511727800001494E4900D11F046
:10112000A3F0900CFFE07004A3E06401900CFF704A
:1011300008F0A3F07F250214A3E4021429900CFF09
:10114000E07002A3E06011900D12E004F0700690D0
:101150000D11E004F00214A6900CD0E0FBA3E0FA1D
:10116000A3E0F912015EFF0214A3900D09E4F0A3BD
:1011700004F0E4900D03F0A3F0A3F0A3F0900CFFB3
:10118000E07004A3E0640160030213FE900D16F00A
:10119000A37404F0900D11E0FEA3E0FF64024E7012
:1011A00026900D16F0A37402F0900D13E0FBA3E45B
:1011B00075F001120209A9F0FA12015EFD900CFD12
:1011C000E4F0A3EDF08021EF64014E900D13E0FBFD
:1011D000A3E475F002120209A9F0FA12021FFF90AF
:1011E0000CFDE5F0F0A3EFF0900D16E0FFA3E0900A
:1011F0000CFBCFF0A3EFF0D3900CFCE09400900C2C
:10120000FBE09400500302131C900D16A3E014257C
:10121000E025E0FD740F7E00A805088005C333CEED
:1012200033CED8F9FF900CFDE05EFEA3E05FA80589
:10123000088005CEC313CE13D8F9FF900CFBE0FC59
:10124000A3E0FD240BF582740D3CF583EFF0740BE5
:101250002DF582740D3CF583E0FFC3940A402BEF1B
:10126000D3940F5025900D09E07002A3E07E5760E3
:10127000027E37EE2FFF900CFBE0FCA3E0240BF581
:1012800082740D3CF583EFF08021900CFBE0FEA30F
:10129000E0FF240BF582740D3EF583E02430FD74ED
:1012A0000B2FF582740D3EF583EDF0900CFBE0FE04
:1012B000A3E0240BF582740D3EF583E0B4302A9050
:1012C0000D03E07002A3E07010900D06E004F070D2
:1012D00026900D05E004F0801E900D04E004F070EF
:1012E00006900D03E004F0800E900D04E004F07011
:1012F00006900D03E004F0900CFEE0C4F8540FC813
:1013000068F0900CFDE0C454F048F0900CFCE02430
:10131000FFF0900CFBE034FFF00211F7900D16E0A7
:10132000FEA3E0FF240CF582740D3EF583E4F090FB
:101330000CFFF0A3F0900D07E07002A3E07008909E
:101340000D07EEF0A3EFF0900D03E0FEA3E0FFC366
:10135000900D08E09F900D07E09E4070E4900CFB1C
:10136000F0A3F0900D03E0FEA3E0FFC3900D08E0B2
:101370009FFF900D07E09EFEC3900CFCE09F900C39
:10138000FBE09E50157F30126F97900CFCE004F04C
:1013900070D1900CFBE004F080C9900D03E0FFA336
:1013A000E0900CFBCFF0A3EFF0900CFBE0FEA3E08D
:1013B000FFD39400EE94004057126F8B900CFCE02A
:1013C00024FFF0900CFBE034FFF080DD900D03E093
:1013D000FFA3E0900CFBCFF0A3EFF0900CFBE0FE3E
:1013E000A3E0FFD39400EE94004025126F8B900C85
:1013F000FCE024FFF0900CFBE034FFF080DD900C6B
:10140000D0E0FBA3E0FAA3E0F912015EFF126F97B0
:10141000E4900D07F0A3F0A38051900CFFE070045E
:10142000A3E064017009900D01F0A304F0807790AF
:101430000CD0E0FBA3E0FAA3E0F912015EFF8063A9
:10144000900D01E07004A3E06401900CD07021E0E5
:10145000FBA3E0FAA3E0F912015E24D0FEE434FF1E
:10146000900D07F0A3CEF0E4900D01F0A3F08036CC
:10147000E0FBA3E0FAA3E0F912015EFF80257F0DF7
:10148000126F97900CD0E0FBA3E0FAA3E0F91201F1
:101490005EFF800F900CD0E0FBA3E0FAA3E0F9120E
:1014A000015EFF126F97900CD0E0FBA3E0FAA3E07F
:1014B0002401F9E43AFA900CD0EBF0A3EAF0A3E9A6
:1014C000F00210C222E59620E7FB75960EE4F59730
:1014D000E59620E7FB759691E59620E7FB900CCF0B
:1014E000E597F0900F21E0B40513E59620E7FBE4C3
:1014F000F596900F18E0F597E4900F21F0900CCF3F
:10150000E0FF30E210E59620E7FB759611E4F597D1
:10151000900F21F022EF30E41BE59620E7FB759653
:1015200011759708E59620E7FB759611759780E48D
:10153000900F21F0900F21E06003021631900CCF44
:10154000E020E0030216317B017A0F79157D087CDB
:10155000007F20126C6C900F18E0FE900F17E07C5B
:10156000002400FFEC3EF0A3EFF0900F1AE0FE9095
:101570000F19E02400FFEC3EF0A3EFF0900F1CE009
:10158000FE900F1BE02400FFEC3EF0A3EFF0900F65
:1015900015E0547F64217035A3E024FE601B1460C5
:1015A0002224FA600F14601614601D240A707F1242
:1015B000706F807D1270BA80781279E5807312782E
:1015C00015806E1279E680691279E78064900F16B3
:1015D000E0B40C0050589015DDF82828730216016D
:1015E00002160602162E02160B02162E0216100204
:1015F000161502162E02161A02161F0216240216BD
:10160000291252EC802B1265BE80261264228021A2
:10161000126F3A801C1238F880171266C6801212B8
:1016200064AD800D126A048008127316800312776D
:1016300050900F21E064016003021704900CCFE08A
:1016400030E103021704E59620E7FB759691E596D5
:1016500020E7FB900CCFE597F0E030E40630E003A4
:10166000021704900CCF7402F0C3900F20E0944056
:10167000900F1FE09400403C900F12E0FBA3E0FAB3
:10168000A3E0F97D407C007F20126E8F900F13E461
:1016900075F0401201F3900F20E024C0F0900F1F6E
:1016A000E034FFF0900F1EE02440F0900F1DE03476
:1016B00000F08024900F1FE0FCA3E0FD900F12E0EB
:1016C000FBA3E0FAA3E0F97F20126E8F900CCFE02D
:1016D0004408F0E4900F21F0900F1BE0FEA3E0FF20
:1016E000A3E0B50611A3E0B5070C900CCFE04408C9
:1016F000F0E4900F21F0E59620E7FB759611900C31
:10170000CFE0F597900F21E0640260030217E6E551
:101710009620E7FB759691E59620E7FB900CCFE5C8
:1017200097F0E020E0030217E67440F0C3900F202A
:10173000E09440900F1FE09400403C900F12E0FBBB
:10174000A3E0FAA3E0F97D407C007F20126C6C904E
:101750000F13E475F0401201F3900F20E024C0F065
:10176000900F1FE034FFF0900F1EE02440F0900F28
:101770001DE03400F0801C900F1FE0FCA3E0FD9002
:101780000F127F20126C64900CCFE04408F0E490BC
:101790000F21F0900F1BE0FEA3E0FFA3E0B50611C0
:1017A000A3E0B5070C900CCFE04408F0E4900F21C3
:1017B000F0900F21E07019900F16E0B40912900F0D
:1017C00012E0FBA3E0FAA3E0F912015EFF126D80C4
:1017D000900F21E064046005E59620E7FB75961103
:1017E000900CCFE0F59722900C71EFF0A3E0FCA3F2
:1017F000E0FDA3E0FEA3E0FF900B5C1203D3E4FF47
:101800001273C9900C79EFF054FEFDE4FF12757A63
:10181000900C71E06416706D7F16127102900C7856
:10182000E0547024F0602024D0602724F0602E243F
:10183000F0603524F0603C24707043900C7A7401A1
:10184000F0A374F4F0803E900C7AE4F0A374FAF004
:101850008033900C7AE4F0A374C8F08028900C7A5E
:10186000E4F0A37464F0801D900C7AE4F0A3743269
:10187000F08012900C7AE4F0A37419F08007E490E1
:101880000C7AF0A3F0900C7AE0FEA3E0FBAA06E449
:10189000F9F8900C72E0FCA3E0FDA3E0FEA3E0FFEA
:1018A0001202F4900C821203D3900C82E0FCA3E0AD
:1018B000FDA3E0FEA3E0FF78061203ADEE543FFE69
:1018C000900C7CEEF0A3EFF0900C7CE0FCA3E0FD2C
:1018D000AE047806C333CE33CED8F92DFFEC3EFEEE
:1018E000900C7EF0A3EFF0E4FCFD900C82E0F8A3F6
:1018F000E0F9A3E0FAA3E0FBD312039C401C900C98
:101900007FE02441F0900C7EE03400F0900C7DE00C
:1019100004F07006900C7CE004F0900C82A3A3E02D
:10192000FEA3E0FFC3900C7FE09FF0900C7EE09E52
:10193000F0900C7CE0FEA3E0FBAA06C3900C7FE0D5
:101940009421900C7EE09400401C900C7DE024FFDC
:10195000F0900C7CE034FFF0900C7FE024DFF090FE
:101960000C7EE034FFF0C3900C7FE09420900C7E5E
:10197000E094004011EB1B70011AA3E024E0F0900A
:101980000C7EE034FFF0900C7EE0FEA3E0FFC394F9
:1019900020EE940050A5EF9410EE94004010E02447
:1019A000E0F0900C7EE034FFF0EB1B70011A900C1D
:1019B0007EE0FEA3E0FFC3900C7DE09FFF900C7CD7
:1019C000E09E900C80F0A3EFF0900C7FE02BFF9056
:1019D0000C7EE03AAD07FC900C71E064167047EDA8
:1019E000AE047806CEC313CE13D8F9540FFF900C73
:1019F00078E054F04FF0900C80E0FAA3E0FBEA545A
:101A000003FFAE05EE25E025E054FC4F900C77F087
:101A1000900C76EBF07B017A0C7976900CC1740314
:101A2000F07F16126AE3900B5BE07003021ADD7F11
:101A300012127102900C78E054FEF0900C77E05492
:101A40003FF04440F07B017A0C7976900CC174032E
:101A5000F07F12126AE37B017A0C79767D037F14A2
:101A600012710A900C77E04408126AD47F017E005C
:101A70001276F57F101273C9EF5407900C86F09020
:101A80000C77E054F7126AD4900C86E0FFD39401EF
:101A90004005EF94064046E4900C7CF0A3F0900CD7
:101AA0007DE004F07006900C7CE004F0900C77E090
:101AB000547F126AD4900C77E04480126AD47F0A73
:101AC0007E001276F57F0E1273C9EF20E10FC390EE
:101AD0000C7DE09403900C7CE0940040C1900C7964
:101AE000E0FDE4FF02757A900C82EBF0A3EAF0A32C
:101AF000E9F0E4900C90F0900B5AE0547FF07F8F67
:101B00001276B01279B17D407F1A12757A7D3F7FCF
:101B10000D12757A7F807E001271927F8F1276B0DF
:101B2000E4900B59F0A3F07F1BFE127192900B5AB8
:101B3000E054176003021C22900B5AE020E30302DA
:101B40001DAC7B017A0E79ED7F01127968900EED64
:101B5000E054F81313543FFF7E00900C86EEF0A380
:101B6000EFF0D39420EE94004009900C86E4F0A3AB
:101B70007420F0900C86A3E0FF900C82E0FBA3E0C1
:101B8000FAA3E02424F9E43AFAEF120199900C87C1
:101B9000E02404F0900C86E03400F0E0FEA3E0784E
:101BA00003C333CE33CED8F9F0EE900C86F0E0FCD0
:101BB000A3E0FDEC54034440900C8AF0EDA3F090B8
:101BC0000C86E0FEA3E07803CEC313CE13D8F9F061
:101BD000EE900C86F07B017A0C798A900CC174022D
:101BE000F07F1A126AE3E4900B59F0A3F07B0190A6
:101BF0000C8D04F0A3740EF0A374EEF0900C87E04B
:101C000024FF8058C3900C87E09412900C86E094D7
:101C10000040537F067E80127192900B5AE054066A
:101C20006009900C9074FFF0021DAC7F1C1273C908
:101C3000900C85EFF0900B59E0547FF0900C8DE004
:101C4000FBA3E0FAA3E0F97F12127968900C8EE40E
:101C500075F0121201F3900C87E024EEF0900C86E0
:101C6000E034FFF0809E7F407E00127192900B5A0C
:101C7000E054157007900C8804F08005E4900C88FF
:101C8000F07F9F1276B07F1C1273C9EF541F900C27
:101C900085F06054E0FFFDC3900C87E09DF0900C50
:101CA00086E09400F0900C8DE0FBA3E0FAA3E0F94D
:101CB000127968E4900C89F0FF900C82E0FBA3E0BD
:101CC000FAA3E02424F9E43AFA12015EFEEFC39E7F
:101CD000501674EF2FF582E4340EF583E070069011
:101CE0000C89E004F00F80D17D377F0D12757A7F6B
:101CF000807E001271927F8F1276B07D207F1B1242
:101D0000757AE4900B59F0A3F07F5FFE1271927F19
:101D10001C1273C9EF541FFF7003021DAC7B017AC4
:101D20000F790F127968900C82E0FBA3E0FAA3E030
:101D30002424F9E43AFA12015EFD900C957401F046
:101D4000A3740EF0A374EDF0A37401F0A3740EF06D
:101D5000A374EFF0A37401F0A3740FF0A3740FF059
:101D6000900C82A3E0FAA3E0F9124C1F7F0F1273CC
:101D7000C9900C82E0FBA3E0FAA3E02427F9E43A3F
:101D8000FAEF120199900C88E0701B900C82E0FB36
:101D9000A3E0FAA3E02424F9E43AFA12015EFF90EA
:101DA0000C89E0B50706900C907401F0E4FD7F1AF1
:101DB00012757A900C90E0FF22900C621203D312FD
:101DC00078CF7F017E001276F5900C667455F0A3F3
:101DD00074AAF0E4A3F0A374FFF07B017A0C796697
:101DE000900CC17404F07F16126AE37E007F047DBC
:101DF000007B017A0C79661205E27B017A0C796628
:101E00007D047F1612710A900C66E0FFB4550EA394
:101E1000E0B4AA09A3E07005A3E0F460257BFF7A93
:101E2000657937900CD3EFF0900C67E0900CD4F00C
:101E3000900C68E0900CD5F0900C69E0900CD6F016
:101E4000803CC2A17F017E001276F5D2A17F017E87
:101E5000001276F57B017A0C79667D047F1612718B
:101E60000A900C66E06455600FA3E064AA6009A3C1
:101E7000E06005A3E0B4FF0B7BFF7A65794C12109C
:101E80008B803EE4900B59F0A3F07D207F0D1275FE
:101E90007A7D027F1E12757A7B017A0C7966900C2E
:101EA000C17404F07F1F126AE37F921276B07F0044
:101EB0007E20127192900B59E0B4FF0AA3E0B4FFA8
:101EC000057E007F0122E4900B59F0A3F0124E0F23
:101ED0007F841276B012798DEF24C8601C24E860EC
:101EE0002614602324FC601F24257023E4900B5BE0
:101EF000F07BFF7A65795B8024900B5B7401F07B4B
:101F0000FF7A6579718016900B5B7402F08016126F
:101F1000798D900CD3EFF07BFF7A65798712108B67
:101F20007E007F0F221275767D067F0112757A7D05
:101F3000F07F0212757A7D097F0A12757A7D087F1B
:101F40000A12757A900C6874E0F0900C6774D8F0FF
:101F5000900C66744FF07B017A0C7966900CC1741A
:101F600003F07F16126AE37D027F0B12757A900CE4
:101F7000667401F07403F0A3743FF0A37420F07B47
:101F8000017A0C7966900CC17403F07F15126AE334
:101F90007D377F0D12757A900C667483F0A304F080
:101FA000A3740AF07A0C7966126AD97BFF7A657994
:101FB0009A12108B900C66740CF0E4A3F0A3F07BE3
:101FC000017A0C7966900CC17403F07F12126AE3F7
:101FD000E4FF1273FB900C62E0FCA3E0FDA3E0FEC3
:101FE000A3E0FF900C721203D37F161217E77F1441
:101FF0007E001276F57F0E1273C9900C66EFF0200A
:10200000E0057E007F0222900C66E020E1057E0064
:102010007F0322122BB2900C6AEEF0A3EFF0900C2B
:102020006AE0FAA3E0FE3395E0A3F0A3CEF0900CB3
:102030006CE0FCA3E0FDFFAE041201AB900C6CEE73
:10204000F0A3EFF0EAFF3395E0FEA3F0FCA3EFF07E
:10205000FD1201AB900C6EEEF0A3EFF0900C6DE072
:102060002FFF900C6CE03EFE900C6AF0A3EFF0D3D3
:102070009400EE940240057E007F0E22E4FEFF22D3
:10208000900F3DEEF0A3EFF0A3EBF0A3EAF0A3E98D
:10209000F0E4FFA3F0A3F0FEFD900F3EE024F090EB
:1020A0000F3DE034D8C364809480400FA3E024F057
:1020B000F0900F3DE034D8F00F80DE900F3EE0242A
:1020C00018900F3DE034FCC3648094804014A3E07A
:1020D0002418F0900F3DE034FCF0900F42E004F043
:1020E00080D9900F3EE0249C900F3DE034FFC36404
:1020F0008094804014A3E0249CF0900F3DE034FFD6
:10210000F0900F43E004F080D9900F3EE024F69069
:102110000F3DE034FFC364809480400FA3E024F6B9
:10212000F0900F3DE034FFF00E80DE900F3EE02493
:10213000FF900F3DE034FFC364809480400FA3E024
:1021400024FFF0900F3DE034FFF00D80DEEF7003D0
:102150000221DA2430FF900F3FE0FBA3E0FAA3E076
:10216000F9EF120199900F42E02430FF900F3FE009
:10217000FBA3E0FAA3E02401F9E43AFAEF12019993
:10218000900F43E02430FF900F3FE0FBA3E0FAA361
:10219000E02402F9E43AFAEF120199EE2430FF90BC
:1021A0000F3FE0FBA3E0FAA3E02403F9E43AFAEFDF
:1021B000120199ED2430FF900F3FE0FBA3E0FAA35A
:1021C000E02404F9E43AFAEF120199900F3FE0FBA2
:1021D000A3E0FAA3E0240502230D900F42E0606C17
:1021E0002430FF900F3FE0FBA3E0FAA3E0F9EF12E9
:1021F0000199900F43E02430FF900F3FE0FBA3E0F4
:10220000FAA3E02401F9E43AFAEF120199EE24303E
:10221000FF900F3FE0FBA3E0FAA3E02402F9E43AC9
:10222000FAEF120199ED2430FF900F3FE0FBA3E09D
:10223000FAA3E02403F9E43AFAEF120199900F3F70
:10224000E0FBA3E0FAA3E0240402230D900F43E097
:1022500060502430FF900F3FE0FBA3E0FAA3E0F9C9
:10226000EF120199EE2430FF900F3FE0FBA3E0FA5C
:10227000A3E02401F9E43AFAEF120199ED2430FFCA
:10228000900F3FE0FBA3E0FAA3E02402F9E43AFA5E
:10229000EF120199900F3FE0FBA3E0FAA3E02403C3
:1022A000806BEE60382430FF900F3FE0FBA3E0FA34
:1022B000A3E0F9EF120199ED2430FF900F3FE0FB0E
:1022C000A3E0FAA3E02401F9E43AFAEF12019990AD
:1022D0000F3FE0FBA3E0FAA3E024028030ED6011A1
:1022E0002430FF900F3FE0FBA3E0FAA3E0F9EF807A
:1022F0000D900F3FE0FBA3E0FAA3E0F97430120168
:1023000099900F3FE0FBA3E0FAA3E02401F9E43A3F
:10231000FAE412019922900C68EBF0A3EAF0A3E929
:10232000F0A3EDF0E4900C74F0A3F0A3F0A3F09010
:102330000C7AF0A37403F0E4900B59F0A3F07F8FB4
:102340001276B0E4900C7AF0900C6BE0FF900C7A6F
:10235000E0C39F504D900C68E0FBA3E0FAA3E0F9C6
:10236000900C7AE0FF75F028A4F582E92582F9EA5D
:1023700035F0FAE4F5F012024AEF75F028A4FF9068
:102380000C68E0FBA3E0FAA3E02FF9EA35F0FAE9E4
:102390002424F9E43AFAE4120199900C7AE004F06A
:1023A00080A6E4900B59F0A3F0900C6CE0FBA3E046
:1023B000FAA3E0F9A3E0FD122F517F2C7E011279E0
:1023C00007E4900B59F0A3F0900C70E0FF126999AC
:1023D000E4900C76F0A3F07F01FEFDFC900C70E021
:1023E000F9F81203C0900C78EEF0A3EFF0900C6BAC
:1023F000E0FD900C74E0FEA3E0FFC39DEE9400406E
:10240000030224DA7C007D281201AB900C68E0FB0B
:10241000A3E0FAA3E02FF9EA3EFA126C02EF14608F
:102420001424027067900C77E004F0705F900C76D3
:10243000E004F08057900C6FE0FF7E00C006C007FC
:10244000900C74E0FEA3E0FF7C007D281201AB90AD
:102450000C68E0FBA3E0FAA3E02FF9EA3EFAE924D6
:1024600004F9E43AA801FCAD03900C6CE0FBA3E096
:10247000FAA3E0F9D007D0061205BEEF700E900C5B
:1024800075E004F07006900C74E004F0900C79E0B4
:1024900024FFF0900C78E034FFF0E4900B59F0A3A7
:1024A000F0900C71A3E0FAA3E0F9120405900C7C03
:1024B000EFF0900C78E07002A3E0600B900C7CE0F1
:1024C00060057F991276B0900C78E07002A3E0600E
:1024D00009900C7CE060030223ED900C7BE014F08B
:1024E000900C76E07002A3E0607DE47F01FEFDFCCD
:1024F000900C70E0F9F81203C0E47B04FAF9F812CA
:1025000002F4A804A905AA06AB07900C76E0FEA386
:10251000E0FFE4FCFDD312039C500A900C70E00431
:10252000F07F9A803DE47F01FEFDFC900C70E0F9A5
:10253000F81203C0E47B08FAF9F81202F4A804A91F
:1025400005AA06AB07900C76E0FEA3E0FFE4FCFDD5
:10255000D312039C400A900C70E014F07F9C800220
:102560007F9B1276B08005E4900C7BF0900C6BE0C2
:10257000FFC3900C75E09F900C74E094005018908D
:102580000C7BE06012900C71A3E0FAA3E0F9120456
:1025900005EF60030223D0900C74E0FEA3E0FF225D
:1025A000900C64EBF0A3EAF0A3E9F0A3EDF0E49063
:1025B0000C6DF0900C80740AF0A37432F012714A22
:1025C000C292D29312799D900C68E0FFA3E0FBA326
:1025D000E0FAA3E0F9A3E0900C89F0124B24D29228
:1025E000D2937F047E001276F5127862125C8B9093
:1025F0000C7EEFF0706D7B01900C8904F0A3740CDD
:10260000F0A37476F0A37408F012411B900C64E000
:10261000FBA3E0FAA3E02424F9E43AFA74081201D7
:1026200099900C64E0FBA3E0FAA3E02404F9E43AF7
:10263000FA900CD3EBF0A3EAF0A3E9F0900C64A3BA
:10264000E0FAA3E02424F9E43AFA12015E900CD6F1
:10265000F07B017A0C796E127219900C6D7401F096
:102660000227EB900C7EE0B4FD08E4900C6DF002C4
:1026700027EB900C8274FFF0A37479F0A374A7F099
:10268000900C7F7402F0900C67E070030227EB90CF
:102690000C80E0FF900C7FE0C39F40030227EB908B
:1026A0000C81E0FF14F0EF70030227EB12714AC2B5
:1026B00092D293900C82A3E0FAA3E0F9120405D21F
:1026C00092D2937F047E001276F5127862125C8BB0
:1026D000900C7EEFF0601424037003022790240214
:1026E00060030227A7900C820227D7900C897401FF
:1026F000F0A3740CF0A37476F0A37408F07B0112BD
:10270000411B900C6DE075F028A4FFAEF0900C64B6
:10271000E0FBA3E0FAA3E02FF9EA3EFAE92424F96A
:10272000E43AFA7408120199900C64E0FBA3E0FA11
:10273000A3E02FF9EA3EFAE92404F9E43AFA900C0E
:10274000D3EBF0A3EAF0A3E9F0900C64A3E0FAA3C2
:10275000E02FF9EA3EFAE92424F9E43AFA12015E9C
:10276000900CD6F07B017A0C796E127219900C6D78
:10277000E004F0900C67E014F0900C7FE014F0900F
:102780000C8274FFF0A37479F0A374A2F002268681
:10279000900C8274FFF0A37479F0A374A2F0900CF3
:1027A0007FE014F0022686900C82E0FBA3E0FAA3FF
:1027B000E0F9EB8A838982F4700A74986582700468
:1027C00074796583900C82600E74FFF0A37479F0C5
:1027D000A37498F002268674FFF0A37479F0A374B2
:1027E000A7F0900C7FE004F0022686900C6DE0FFCD
:1027F00022011000010A00011101500F24BFAFA7F0
:10280000A3A1A0B0B8BCBE41888A642082480DADA7
:10281000FFFFFFFFFFFFFFFF60400D2A00000000E9
:1028200000000000000000000000000000000000A8
:102830000000000000000000000000000000000098
:102840000000000000000000000000000000000088
:10285000000000000000000000000000490F34FFED
:102860007F67FF7F6CFF7F78430F210003034C0ECF
:102870007605FF74F50000000000000000500E61B6
:1028800002FF77BC00000000000000000000000014
:10289000410E7100440B4306010001410B4A044103
:1028A0000B5403410B5332440B4F000DC65E4400E2
:1028B00008000E2612420B3A0000420B180190420B
:1028C0000B480000410B41024100000041000100A3
:1028D00041000200410B5800410B5500420B5900CA
:1028E0000060FC0B600000010203040506070809F4
:1028F0000A0B0C0D0E0F10111213141516171819C0
:102900001A1B1C1D1E1F20212223242526272829AF
:102910002A2B2C2D2E2F303132333435363738399F
:102920003A3B3C3D3E3F404142434445464748498F
:102930004A4B4C4D4E4F505152535455565758597F
:102940005A5B5C5D5E5F606162636465666768696F
:102950006A6B6C6D6E6F707172737475767778795F
:102960007A7B7C7D7E7F808182838485868788894F
:102970008A8B8C8D8E8F909192939495969798993F
:102980009A9B9C9D9E9FA0A1A2A3A4A5A6A7A8A92F
:10299000AAABACADAEAFB0B1B2B3B4B5B6B7B8B91F
:1029A000BABBBCBDBEBFC0C1C2C3C4C5C6C7C8C90F
:1029B000CACBCCCDCECFD0D1D2D3D4D5D6D7D8D9FF
:1029C000DADBDCDDDEDFE0E1E2E3E4E5E6E7E8E9EF
:1029D000EAEBECEDEEEFF0F1F2F3F4F5F6F7F8F9DF
:1029E000FA00E4900C62F0900E727440F0A374014F
:1029F000F0A3740DF0A3746CF0900D6C7444F0A30C
:102A00007440F0900E1FE0640170527F0112725A00
:102A100012376BE4900002F0900B16F0A3F0EF7009
:102A2000377B01900C6C04F0A3740BF0A3741AF0C4
:102A3000E4A3F0900B4AE0900C70F0A374FFF0A3B5
:102A40007475F0A374F3F07A0179167D40122316A1
:102A5000900B16EEF0A3EFF0E4FF12746290000208
:102A6000E0FFD3900B17E09F900B16E0940050030B
:102A7000022B86900002E0FD75F028A4243AF5822E
:102A8000E5F03401F583E0FE240A900D6DF0EE24AC
:102A900002900D73F075F028EDA42418F582E5F08E
:102AA0003401F583E0900D74F0900002E075F02899
:102AB000A42419F582E5F03401F583E0900D75F05A
:102AC000EF75F028A4241AF9740135F0FA7B01C0DF
:102AD00003900CD3EBF0A3740DF0A37476F0900088
:102AE00002E075F028A4243AF582E5F03401F5837C
:102AF000E0900CD6F0D003127219900002E075F04D
:102B000028A4243DF582E5F03401F583E0900D6FB3
:102B1000F0900B3DE0FEA3E07802C333CE33CED875
:102B2000F9FBAA06240DF58274003AF583A3A3A34A
:102B3000E0FF900D70EFF0740D2BF58274003AF504
:102B400083E0FCA3E0FDA3E0FEA3E0FF780812030E
:102B5000AD900D71EFF0900B3DE0FEA3E07802C365
:102B600033CE33CED8F9240DF58274003EF583E0E0
:102B7000FCA3E0FDA3E0FEA3E0FF78101203AD90FC
:102B80000D72EFF0800B900D6D7405F0E4900D70F8
:102B9000F0900B16E0FEA3E0FF4E600A900002E00A
:102BA000FEC3EF9E8001E4900D6EF0900002E00401
:102BB000F022E4FF1273C9900C7AEFF07B017A0CDB
:102BC00079767D037F1412710A900C76E0900C796F
:102BD000F054CF900C76F07B017A0C7976126ADB98
:102BE0001275767F961276B07F017E001276F57FA1
:102BF000971276B07D017F1112757A7F027E0012E6
:102C000076F57F871276B07F147E001279077F19E0
:102C10001273C9900C74EFF05480FF3395E04F604D
:102C200006E0547FFF8009900C74E0547FF404FFA9
:102C3000900C74EFF07D027F1112757A7F027E0096
:102C40001276F57F871276B07F147E001279077FA7
:102C5000191273C9900C75EFF05480FF3395E04F53
:102C60006006E0547FFF8009900C75E0547FF40407
:102C7000FF900C75EFF07D03E4FF12757A7F9612DA
:102C800076B07F017E001276F57F971276B07D01D7
:102C90007F1112757A7F027E001276F57F87127699
:102CA000B07F147E001279077F191273C9900C73DC
:102CB000EFF05480FF3395E04F6006E0547FFF80D3
:102CC00009900C73E0547FF404FF900C73EFF0A3B1
:102CD000E0FD3395E0FCEF3395E0FEC3EF9DFFEEA2
:102CE0009C900C71F0A3EFF07D027F1112757A7F3A
:102CF000027E001276F57F871276B07F147E001276
:102D000079077F191273C9900C73EFF07F961276D2
:102D1000B0900C73E0FF5480FD3395E04D6006EFFA
:102D2000547FFF8009900C73E0547FF404FF900CF3
:102D300073EFF0900C75E0FEC3EF9EFF900C73F004
:102D4000EFFE900C72E0FDEDFF900C71EEF0A3EF42
:102D5000F07B017A0C79767D037F1412710A900C56
:102D600079E0900C76F07B017A0C7976126ADB9030
:102D70000C7AE0FDE4FF12757A900C71E0FEA3E09E
:102D8000FF22FDF0900C8DE0FF3395E0FEEF25E093
:102D9000FFEE33FE74822FF9740E3EFA7B01900C25
:102DA000A0EBF0A3EAF0A3E9F0900CA0E0FBA3E015
:102DB000FAA3E0F9E4120199900CA0E0FBA3E0FA79
:102DC000A3E02402F9E43AFAE4120199900CA0E09D
:102DD000FBA3E0FAA3E02401F9E43AFA7408120133
:102DE00099900CA0E0FBA3E0FAA3E02403F9E43AF5
:102DF000FA7408120199ED900CA030E70FE0FBA3E4
:102E0000E0FAA3E0F912015E4480800DE0FBA3E04C
:102E1000FAA3E0F912015E4440120199ED900CA072
:102E200030E60FE0FBA3E0FAA3E0F912015E4420D4
:102E3000800DE0FBA3E0FAA3E0F912015E4410125A
:102E40000199ED900CA030E50FE0FBA3E0FAA3E0C0
:102E5000F912015E4408800DE0FBA3E0FAA3E0F95B
:102E600012015E4404120199ED900CA030E40FE0D1
:102E7000FBA3E0FAA3E0F912015E4402800DE0FB3F
:102E8000A3E0FAA3E0F912015E4401120199ED906A
:102E90000CA030E314E0FBA3E0FAA3E02402F9E481
:102EA0003AFA12015E44808012E0FBA3E0FAA3E04C
:102EB0002402F9E43AFA12015E4440120199ED90BD
:102EC0000CA030E214E0FBA3E0FAA3E02402F9E452
:102ED0003AFA12015E44208012E0FBA3E0FAA3E07C
:102EE0002402F9E43AFA12015E4410120199ED90BD
:102EF0000CA030E114E0FBA3E0FAA3E02402F9E423
:102F00003AFA12015E44088012E0FBA3E0FAA3E063
:102F10002402F9E43AFA12015E4404120199ED9098
:102F20000CA030E014E0FBA3E0FAA3E02402F9E4F3
:102F30003AFA12015E44028012E0FBA3E0FAA3E039
:102F40002402F9E43AFA12015E44011201997F0267
:102F500022900C7DEBF0A3EAF0A3E9F0A3EDF0A33F
:102F60007412F07F8F1276B0784D768F087690903D
:102F70000C80E0FD2403FFE433FEEF7804CEA2E7EB
:102F800013CE13D8F87821F6ED2403540FC454F06F
:102F9000440B08F6900C80E033333354F8FFF09084
:102FA0000EEAE025E0540E44A008F6087612900CD4
:102FB00080E0FEC4540F08F6EEC454F008F67E0517
:102FC000EFC39408403A74212EF8C000E6FD900C3F
:102FD0007DE0FBA3E0FAA3E0F912015EFCC4540F0C
:102FE0004DD000F60EECC454F0FD74212EF8A60569
:102FF00074F82FFF900C7EE475F0011201F380C08D
:1030000074212EF8E6F6900C80E0FF131313541F82
:10301000F0E02406F0900C82E4F0A37400F0A374B6
:1030200021F0900C80E0D3941A50030230E7900B0B
:1030300059E054BFF0900C8A741DF0900C82E0F9B6
:10304000A3E0FAA3E0900C8BC9F0A3EAF0A3E9F0A7
:10305000A3741AF07B007A00794E7D01126CC49043
:103060000C80E024E6F0900C83E475F01A804E901A
:103070000C81E0FF900C80E0D39F40467D0F7C00E8
:103080007F007E40126D22900B59E054BFF0900CEF
:1030900082E0FBA3E0FAA3E0F9900C81E0900CC180
:1030A000F07F1F126AE3900C80E0FFA3E0FEC3EF05
:1030B0009E900C80F0EEFF900C83E48FF01201F3F1
:1030C00080AD7D0F7C007F007E40126D22900C82CF
:1030D000E0FBA3E0FAA3E0F9900C80E0900CC1F0D3
:1030E0007F1F126AE3802E900C8A741DF0900C8270
:1030F000E0F9A3E0FAA3E0900C8BC9F0A3EAF0A3F7
:10310000E9F0900C80E0900C8EF07B007A00794E14
:103110007D01126CC47D0F7C007F807E00026D22D9
:10312000900C64EBF0A3EAF0A3E9F0A3EDF0900CAF
:103130006F740DF0E4900C6EF0900C6BE0FF14F0E7
:10314000EF70030232B3900C6EE060030232B312F0
:10315000714AC292D293D2937F017E001276F51209
:1031600055DB900C6CEFF03395E0FEEF25E0FFEEC1
:1031700033FE74822FF9740E3EFA7B01900C6FE0DF
:10318000FD122D9E900C6CE02FF0900C6FE0A3F0E0
:10319000E4900C6DF0900C64E0FBA3E0FAA3E0F97E
:1031A000900C6DE0FFFD3395E0FCE92DF9EA3CFA67
:1031B00012015EFEEF3395E0FC74712DF582740C04
:1031C0003CF583EEF0900C6CE0FF3395E0FEEF25CC
:1031D000E0FFEE33FE74822FF9740E3EFA7B017429
:1031E000712DF582740C3CF583E0FD122D9E900C40
:1031F0006CE02FF0A3E004F0E0C364809488409575
:10320000900C67E0FD900C79F0900C6C122D87907B
:103210000C6CE02FF0900C67E004F0A3E0FBA3E05F
:10322000FAA3E0F912015EFD900C7AF0900C6C129A
:103230002D87900C6CE02FF0900C69E475F0011272
:1032400001F37B017A0C79707D0B7C001260259074
:103250000C6C126DDC900C6CE02FF07B017A0E7917
:1032600082E0FD3395E0FC12754BD293D292D2935B
:103270007F047E001276F51278627B017A0C797BEE
:103280007D01125C93900C6EEFF0700E900C7BE061
:103290007FFC7001FF900C6EEFF012714AC292D267
:1032A00093D2937F0F7E001276F512729912786294
:1032B000023139900C6EE0FF22900C65EBF0A3EA2E
:1032C000F0A3E9F0900EEC7401F078E87C0EFD902C
:1032D0000C65E0FBA3E0FAA3E0F97E007F04120195
:1032E00016900EE9E07005900EEB04F0900C65E08E
:1032F000FBA3E0FAA3E0F912015E70030233C824D5
:10330000FA70030233A624FE607814605224FD6034
:103310002A24FD600302344CE4900C68F0A374F09E
:10332000F0A374F2F0A3744DF0A37401F0A374043D
:10333000F0E4A3F0A37407F00233EF900C6874017B
:10334000F0A374F0F0A374C2F0A3749BF0A3740212
:10335000F0A37406F0E4A3F0A37427F00233EF9017
:103360000C687401F0A374F0F0A37492F0A374419C
:10337000F0A37403F0A37405F0A314F0A37437F062
:10338000806D900C687402F0A374F0F0A37482F066
:10339000A374E8F0A37403F0A37406F0A37404F01C
:1033A000A3743BF08049900C687402F0A374F0F0B1
:1033B000A37462F0A37435F0A37405F0A37407F04E
:1033C000A3F0A3743FF08027900C687402F0A374FC
:1033D000F0F0A37402F0A374D0F0A37407F0A37408
:1033E0001BF0A37407F0A374FFF0E4900EECF090D0
:1033F0000EE9E025E025E0FF900C68E054F34FF083
:10340000900EEBE07F0060027F01EF25E0FF900C63
:103410006AE054FD4FF07B017A0C7968900CC1741E
:1034200004F07F01126AE37F051273C9EF54F0FFC5
:10343000900C6CE04FFD7F0512757A7B017A0C7958
:103440006D900CC17403F07F07126AE322900C7335
:10345000EBF0A3EAF0A3E9F0EEC313FEEF13FF9045
:103460000C7DEEF0A3EFF04E7007900C7DF0A304FE
:10347000F0E4FF1273C9900C79EFF01275767F09B2
:103480001273C9900C7CEFF07DFF7F0912757A9062
:103490000C79E020E1077F0A7E001276F5E4900CBB
:1034A0007FF0900C7D74FFF5F012020945F0604842
:1034B00012761C900C7AEFF0E0FFC4540FFEEF542C
:1034C0000F2EFF900C80F0900C7FE0FD3395E0FC18
:1034D000D3EF9DEC6480F874809840C6A3E0900C14
:1034E0007FF0900C7AE0FF900C73E0FBA3E0FAA36E
:1034F000E0F9EF12019980AA900C7FE0FF701F9015
:103500000C76E0FBA3E0FAA3E0F974801201999035
:103510000C73E0FBA3E0FAA3E0F9E40235B7EF781F
:1035200003A2E713D8FBFF900C7FE02FF07F0A1275
:1035300073C9900C7BEFF07F051273C9900C7BE090
:10354000FE30E211900C7FE024B5F0EE30E023E095
:103550002405F0801D900C7FE024B9F0EE30E104EA
:10356000E024F6F0900C7BE030E007900C7FE02444
:1035700008F0EF30E71C900C7FE0FF900C7BE0C47C
:103580001313540375F003A4FEC3EF9E900C7FF059
:103590008014900C7BE0C41313540375F003A4FF54
:1035A000900C7FE02FF0900C7FE0FF900C76E0FB1A
:1035B000A3E0FAA3E0F9EF120199900C7CE0FD7F03
:1035C0000912757A900C79E0FDE4FF12757A900C7F
:1035D00079E030E0077F027E001276F522900C68D9
:1035E000EBF0A3EAF0A3E9F0E4900C71F0A3F0781B
:1035F0004D768F0876917821F60876550876C2AF19
:1036000005EFC4333354C0FF08F6900C6CE0FE1392
:1036100013543F4FF6EEC4333354C0FF08F6A3E013
:10362000FE1313543F4FF6EEC4333354C0FF08F675
:10363000E92425F9E43AFA12015EFE1313543F4FD0
:10364000F6EEC4333354C0FF08F6900C68E0FBA3D9
:10365000E0FAA3E02426F9E43AFA12015EFE13131D
:10366000543F4FF6EEC4333354C008F6E4900B5980
:10367000F0A3F07F8F1276B0900C8A741DF0A3E453
:10368000F0A37400F0A37421F0A37408F07B007A17
:1036900000794E7D01126CC47F807E00127192E42D
:1036A000900B59F0A3F07F8F1276B07F5E7E801270
:1036B0007192900B5AE030E333900C6EE0FBA3E084
:1036C000FAA3E0F97F01127968900C6EE0FBA3E0A9
:1036D000FAA3E0F912015E4480120199900C6EE0A9
:1036E000FBA3E0FAA3E0F912015EFF22900B5AE07F
:1036F000541F600F7F1C1273C9EF541F900C72F09F
:103700007F0822900B59E030E731900C6EE0FBA36C
:10371000E0FAA3E0F97F12127968900C6FE475F07B
:10372000121201F3900C71E02412F0900B59E05446
:103730007FF07F5E7E8012719280C8E4900B59F01A
:10374000A3F07F1C1273C9EF541FFF900C72F0900E
:103750000C6EE0FBA3E0FAA3E0F9127968900C721A
:10376000E0FF900C71E02FF07F0022900B18E0FC3E
:10377000A3E0FD24F0FBEC34FFFAD3EB94E8EA94E9
:1037800003401BED2410FFE43CFEEF7806CEC3138C
:10379000CE13D8F9FF7C007D301201AB80167C007F
:1037A0007D30AF03AE021201ABEF7806CEC313CE6D
:1037B00013D8F9FF900B3FEEF0A3EFF0E4FF127483
:1037C00062900B3AE0FEA3E0FFD39414EE94004025
:1037D0000BEF24ECFFEE34FFFE1276F590000CE0C8
:1037E00070037F0A22900B3DA3E0900C69F0900BD0
:1037F00048E0FEA3E0FF900C767401F0A3740CF097
:10380000A3746AF07B017A0C796B12344DE4900C4E
:1038100068F090000CE0FF900B3DE475F0011201A0
:10382000F3FCC3E5F09FEC94004007E4900B3DF0FF
:10383000A3F0900B3DE0FEA3E07802C333CE33CE7D
:10384000D8F9240DF58274003EF583E0FCA3E0FD79
:10385000A3E0FEA3E0FF900C721203D37F161217B1
:10386000E7900B48E0FEA3E0FF900C767401F0A314
:10387000740CF0A3746AF07B017A0C796B12344DEE
:10388000900B3DE0FEA3E024E1F58274003EF58359
:10389000E0FF900C6AE0FED3EF6480F8EE6480985D
:1038A000400F900C68E004F0E0C3943550030238F8
:1038B00012900B3DE0FEA3E024E1F58274003EF59A
:1038C00083E0FF900C6AE0FED3EF6480F8EE648042
:1038D00098501712768CE4900B42F07F01127462BC
:1038E0007F027E001276F57F0022900B427401F079
:1038F000E4FF1274627F0A22900F17E024DF700346
:103900000239E9147003023A072421B40500400388
:10391000023A2190392175F003A4C58325F0C583AF
:10392000730239300239430239690239980239B2D7
:10393000900F1274FFF0A3747CF0A374EAF0907CF3
:10394000EA8066900F1274FFF0A3747CF0A374FCFD
:10395000F0907CFFE493FE907CFEE4937C002400D6
:10396000FFEC3E900F1F023A01900F18E075F00334
:10397000A42434F582E5F0340FF583E0FBA3E0FAEC
:10398000A3E0F9900F12EBF0A3EAF0A3E9F0120123
:103990005EFF900F1FE48069900F1274FFF0A37414
:1039A0007DF0A37405F0907D05E493FF900F1FE474
:1039B000804F900F18E0FF64817066EF900F12B493
:1039C000811074FFF0A3747DF0A37417F0907D173D
:1039D000800E74FFF0A3747DF0A3741EF0907D1E22
:1039E000E493FF900F1FE48018900F1274FFF0A370
:1039F000747DF0A3740EF0907D0EE493FF900F1F82
:103A0000E4F0A3EFF0801D900F1274FFF0A3747D1B
:103A1000F0A37425F0900F1F7402F0A37442F0809D
:103A200003127750900F17E0FF64016013EF6402F8
:103A3000600EEF64036009EF64046004EFB40523D3
:103A4000900F1CE0FFD3900F20E09F900F1FE09499
:103A5000004010900F1BE0700AE0FE900F1FEEF088
:103A6000A3EFF0900F21E064046018E59620E7FBD7
:103A7000759611759740900F217401F0E4900F1D19
:103A8000F0A3F022900C66EBF0A3EAF0A3E9F0E4D7
:103A9000900C6CF0900C66E0FBA3E0FAA3E0242508
:103AA000F9E43AFA900C827401F0A3740CF0A37458
:103AB0006DF0125167EF6008E4900B59F0A3F0220B
:103AC000784D768F087690E47821F608765008765F
:103AD000C6900C69E0FBA3E0FAA3E0F912015EFFD7
:103AE000900C6DE06F08F6E92401F9E43AFA12014E
:103AF0005EFF900C6EE06F08F6900C66E0FBA3E0B2
:103B0000FAA3E02425F9E43AFA12015E08F6900CD3
:103B100066E0FBA3E0FAA3E02426F9E43AFA1201F6
:103B20005E08F67F8F1276B0E4900B59F0A3F09008
:103B30000C8A741DF0A3E4F0A37400F0A37421F0C8
:103B4000A37407F07B007A00794E7D01126CC4E407
:103B5000900B59F0A3F07F5FFE127192900B5AE028
:103B600020E0767F1C1273C9EF540FFFC39403400B
:103B7000027F037B017A0C796F127968900C66E002
:103B8000FBA3E0FAA3E02426F9E43AFA12015EFF6F
:103B9000900C70E06F7038900C66A3E0FAA3E024FC
:103BA00025F9E43AFA12015EFF900C6FE0B5071FA9
:103BB0007F8F1276B0E4900B59F0A3F0900C6A75E9
:103BC000F0021201F3900C6CE0B401157F0022E4C6
:103BD000900B59F0A3F07F0222900C6C7402F0FF5E
:103BE00022E4900B59F0A3F0900C6CE004F0E0C3D9
:103BF00094025003023A947F002212376B900C65B6
:103C0000EFF06003023D161268B8900B16E07002E8
:103C1000A3E07009900C657409F0023D16900E2126
:103C2000E0700CA3E07008A3E07004A3E0602690AD
:103C30000C697401F0A3740EF0A37421F0900B4B87
:103C4000E0FBA3E0FAA3E0F9123A84900C65EFF0F0
:103C50006003023D16900E1FE0FFB401057402F0F0
:103C6000800AEFB40206900E1F7401F0E4900C621B
:103C7000F0A3F0A3F0900E20E0FD7010900C6274A1
:103C8000C0F0900E1FE0FEC45430802BEDB4011341
:103C9000900C627430F0900E1FE0FF25E025E05498
:103CA0000C8014900E20E0FDB40212900C62740C93
:103CB000F0900E1FE05403900C63F08038EDB403D5
:103CC00012900C627403F0900E1FE0FFC433335463
:103CD000C08015900E20E0B40414900C6374C0F002
:103CE000900E1FE0FFC45430900C64F08007E49005
:103CF0000C62F0A3F0900C697401F0A3740CF0A3B3
:103D00007462F0900B4BE0FBA3E0FAA3E0F91250D1
:103D1000A2900C65EFF0E4FF127462900D6C743C9D
:103D2000F0A37404F0900C65E0900D6EF0900E73AB
:103D3000E0FBA3E0FAA3E02401F9E43AFA12015E01
:103D4000900E72F0A37401F0A3740DF0A3746CF0E4
:103D5000027520E4900C62F0900E1FE06401705236
:103D60007F0112725A12376BE4900001F0900B162B
:103D7000F0A3F0EF70377B01900C6C04F0A3740B90
:103D8000F0A3741AF0E4A3F0900B4AE0900C70F0EA
:103D9000A374FFF0A37475F0A374F3F07A0179169D
:103DA0007D40122316900B16EEF0A3EFF0E4FF1205
:103DB0007462900E737401F0A3740DF0A3746CF030
:103DC000900E727440F0900D6C7432F0900B16E00F
:103DD000FEA3E0FF4E600A900001E0FEC3EF9E806C
:103DE00001E4900D6EF0900001E0FFD3900B17E01E
:103DF0009F900B16E094005003023E85900001E076
:103E0000FD75F028A4243AF582E5F03401F583E04D
:103E1000FE2406900D6DF0EE2402900D6FF075F00B
:103E200028EDA42418F582E5F03401F583E0900D27
:103E300070F0900001E075F028A42419F582E5F0F7
:103E40003401F583E0900D71F0EF75F028A4241A89
:103E5000F9740135F0FA7B01C003900CD3EBF0A3A9
:103E6000740DF0A37472F0900001E075F028A424A2
:103E70003AF582E5F03401F583E0900CD6F0D003FA
:103E8000127219800B900D6D7404F0E4900D6FF0B8
:103E9000900001E004F02212376B900C62EFF060AA
:103EA00003023F9D1268B8900B16E07002A3E07009
:103EB00009900C627409F0023F9D900E21E070178A
:103EC000A3E07013A3E0700FA3E0700B7BFF7A6296
:103ED000795E12108B8021900C697401F0A3740E2E
:103EE000F0A37421F0900B4BE0FBA3E0FAA3E0F900
:103EF000123A84900C62EFF0900E1FE024FE6023D3
:103F000024FA605314606524086003023F9D900BFF
:103F10004BE0FBA3E0FAA3E0F9900E20E0FD12567F
:103F2000918042900E20E06010900B4BE0FBA3E0EC
:103F3000FAA3E0F9125A9F801C900C667401F0A35A
:103F4000740EF0A37421F0900B4BE0FBA3E0FAA3F6
:103F5000E0F9124A25800E900B4BE0FBA3E0FAA398
:103F6000E0F9125B44900C62EFF08031900C6674C3
:103F700001F0A3740EF0A37425F0900B4BE0FBA3AB
:103F8000E0FAA3E0F9124D18900C62EFF0900E25C4
:103F9000E0900D6FF0900E26E0900D70F0E4FF12AF
:103FA0007462900D6C7446F0A37405F0900C62E09E
:103FB000900D6EF0900E73E0FBA3E0FAA3E02401F5
:103FC000F9E43AFA12015E900E72F0A37401F0A3C4
:103FD000740DF0A3746CF0027520900F4AEBF0A3FF
:103FE000EAF0A3E9F0A3EDF0E4900F4FF07BFF7A45
:103FF0005D79EC900F4EE0900CD3F012108B900F87
:104000004AE0FBA3E0FAA3E02401F9E43AFA120142
:104010005E900CD3F0900F4AA3E0FAA3E0F91201EE
:104020005E900CD4F07BFF7A5D79F712108B7BFFEA
:104030007A5E7908900F4DE02402900CD3F01210B4
:104040008B900F4AE0FBA3E0FAA3E02403F9E43AE3
:10405000FA12015E900CD3F0900F4AA3E0FAA3E0AD
:104060002402F9E43AFA12015E900CD4F07BFF7A54
:104070005E792212108B7BFF7A5E793012108B9062
:104080000F4DE0FF900F4FE0FEC39F5030900F4A5E
:10409000E0FBA3E0FAA3E02404F9E43AFAEE7E00A0
:1040A00029F9EE3AFA12015E900CD3F07BFF7A5DAB
:1040B00079E412108B900F4FE004F080C27BFF7AFE
:1040C0005D79EA12108B900F4AE0FBA3E0FAA3E0BF
:1040D0002424F9E43AFA12015E900CD3F07BFF7AC3
:1040E0005E793612108B900F4AE0FBA3E0FAA3E052
:1040F0002425F9E43AFA12015E900CD3F0900F4AAD
:10410000A3E0FAA3E02426F9E43AFA12015E900C47
:10411000D4F07BFF7A5E794C02108B7A0C796EE4D6
:10412000FD900C85EBF0A3EAF0A3E9F0A3EDF0908D
:104130000C9A7451F012714AC292D293D2937F01B9
:104140007E001276F51255DB900C8DEFF03395E082
:10415000FEEF25E0FFEE33FE74822FF9740E3EFA77
:104160007B01900C9AE0FD122D9E900C8DE02FF0BB
:10417000900C9AE0900C8FF0E4900C8EF0900C85EF
:10418000E0FBA3E0FAA3E0F9900C8EE0FFFD33958D
:10419000E0FCE92DF9EA3CFA12015EFEEF3395E00E
:1041A000FC74902DF582740C3CF583EEF0900C8D30
:1041B000E0FF3395E0FEEF25E0FFEE33FE74822F43
:1041C000F9740E3EFA7B0174902DF582740C3CF567
:1041D00083E0FD122D9E900C8DE02FF0A3E004F003
:1041E000E0C3648094884095900C88E0900C98120D
:1041F0002D82900C8DE02FF0900C8CE014900C9997
:10420000122D82900C8DE02FF07B017A0C798F7D3E
:104210000B7C00126025900C8D126DDC900C8DE0F3
:104220002FF07B017A0E7982E0FD3395E0FC127568
:104230004BD293D292D293900C8CE075F004A4FFF1
:10424000AEF01276F5127862900C89E0FBA3E0FAEA
:10425000A3E0F9A3E0FD125C9322E4900C62F090DD
:104260000E1FE0640170697F0212725A12376B9060
:104270000C63EFF0E4900000F0126B3B900C63E0F5
:104280006009E4900B16F0A3F08032900E20E090CD
:104290000C68F0A37401F0A3740EF0A37421F090E5
:1042A0000E29E0900C6CF07B017A0179167D4012AA
:1042B00025A0EF3395E0900B16F0A3EFF0E4FF128A
:1042C0007462900B4B7401F0A37401F0A37416F0A8
:1042D000E4900C62F0900C62E0FFC3940C501474F4
:1042E0006C2FF582E4340DF583E4F0900C62E00469
:1042F000F080E2900D6C7440F0A3740DF0E4900D2A
:104300006FF0900000E0FF75F028A4243AF582E5F4
:10431000F03401F583E0900D70F0603AEF75F0280D
:10432000A4241AF9740135F0FA7B01C003900CD370
:10433000EBF0A3740DF0A37471F0900000E075F041
:1043400028A4243AF582E5F03401F583E0900CD6F8
:10435000F0D003127219900B16E0FEA3E0FF4E603E
:104360000E900000E0FEC3EF9E900D6EF08009906D
:104370000D6D7405F0E4A3F0900000E004F0900EE1
:1043800072740DF0A37401F0A3740DF0A3746CF0BB
:10439000027520E4900C63F0900E21E0900C62F026
:1043A00012376B900C63EFF0600302448D1268B813
:1043B000900B16E07002A3E07009900C637409F092
:1043C00002448D900C62E0600302445B7B01900C20
:1043D0006404F0A3740DF0A37470F0900E20E090CC
:1043E0000C67F0900C63E0705E900C62E0C3941E6A
:1043F00050551275F3EF604F900E1FE0FD900C6763
:10440000E0FF04F0900C6CEFF0A37401F0900C64EA
:10441000E0F9A3E0FAA3E0900C6EC9F0A3EAF0A3E0
:10442000E9F0900B4BE0FBA3E0FAA3E0F91235DDD5
:10443000900C63EFF0900C62E004F0900C65E47572
:10444000F0021201F3809C900C62E014F0900B4299
:10445000E0603A900C63740AF08032900E1FE0FD29
:10446000A3E0900C6CF0900C62E0900C6DF0A374E3
:1044700001F0A3740DF0A37470F0900B4BE0FBA35C
:10448000E0FAA3E0F91235DD900C63EFF0E4FF12DF
:104490007462900D6C7438F0900C63E0900D6EF0C7
:1044A000900C62E0FD25E02404900D6DF0900D6FFE
:1044B000EDF0900E727440F0A37401F0A3740DF04F
:1044C000A3746CF0027520900C63EBF0A3EAF0A3E8
:1044D000E9F0E4900C6AF0900C63E0FBA3E0FAA32F
:1044E000E02425F9E43AFA900C827401F0A3740CEC
:1044F000F0A3746BF0125167EF600122784D768F54
:10450000900C6AE0FE7003087690EEB40104784ED9
:104510007691E47821F60876570876C4900C66E028
:10452000FBA3E0FAA3E0F912015EFF900C6BE06FD1
:1045300008F6E92401F9E43AFA12015EFF900C6CE6
:10454000E06F08F6900C63E0FBA3E0FAA3E02425FB
:10455000F9E43AFA12015EFF131313541FFE900C94
:1045600069E0C43354E04E08F6900C63E0FBA3E02E
:10457000FAA3E02426F9E43AFA12015EFE131313BB
:10458000541FFDEFC43354E04D08F6EEC43354E03D
:1045900008F67D367F0D12757A7F8F1276B0E49023
:1045A0000B59F0A3F0900C8A741DF0A3E4F0A374EF
:1045B00000F0A37421F0A37408F07B007A00794E18
:1045C0007D01126CC4900C63125BE9EF60012290D4
:1045D0000C67E475F0021201F3900C6AE004F0E05D
:1045E000C3940250030244D77F0022900C78EDF070
:1045F000900C75EBF0A3EAF0A3E9F02425F9E43A76
:10460000FA900C827401F0A3740CF0A3747DF01284
:104610005167EF6008E4900B59F0A3F022784D76D3
:104620008F087691E47821F60876650876C3900CB9
:1046300078E0C4333354C0FF08F6A3E0FE131354EC
:104640003F4FF6EEC4333354C0FF08F6A3E0FBA39C
:10465000E0FAA3E0F912015EFE900C7DE06EFE131D
:1046600013543F4FF6EEC4333354C0FF08F6E92429
:1046700001F9E43AFA12015EFE900C7EE06EFE1340
:1046800013543F4FF6AF06EFC4333354C0FF08F660
:10469000900C75E0FBA3E0FAA3E02425F9E43AFAD4
:1046A00012015EFE1313543F4FF6EEC4333354C071
:1046B000FF08F6900C75E0FBA3E0FAA3E02426F9CE
:1046C000E43AFA12015EFE1313543F4FF6EEC43380
:1046D0003354C008F67D367F0D12757A7F8F1276BF
:1046E000B0E4900B59F0A3F0900C8A741DF0A3E491
:1046F000F0A37400F0A37421F0A37409F07B007A96
:1047000000794E7D01126CC4900C75125BE9229009
:104710000B41E024FD60481470030247DF2402606F
:1047200003024816E4900007F0FFFEFDFC90000332
:104730001203D3900E1E7402F0120026EF700302D3
:10474000481C127961900007E0FE04F0741D2EF5FC
:1047500082E4340EF583EFF0900B417403F0229065
:104760000003E0FCA3E0FDA3E0FEA3E0FFE4FAF910
:10477000F8EF2401FFEA3EFEE93DFDE83CFC900035
:10478000031203D3E4FF7E80FDFC900003E0F8A356
:10479000E0F9A3E0FAA3E0FBD312038650139000E4
:1047A00007E0FF943F500A900E1EE0FEEFC39E40CC
:1047B00007900B417404F022120026EF605E12791C
:1047C00061900007E0FE04F0741D2EF582E4340EC3
:1047D000F583EFF0E4FFFEFDFC9000030203D37FBE
:1047E00040900D6CE4F0A3DFFC900B417402F0905C
:1047F0000B3C14F0900E1DE075F003A424EAF58242
:10480000E5F03479F583740193FA740293F9120494
:1048100005E4900B3CF0900B417402F022900C7177
:10482000EFF07F051273C9900C731273C5900C7270
:10483000EFF0543CF030E21A900C71E0244BF0E0C1
:10484000D3648094854037E024FBF0A3E04401F07A
:10485000802C900C71E02447F0E0C3648094884081
:1048600009E024F8F0A3E04401F0900C71E0D36477
:104870008094765009E0240AF0A3E04402F0900C02
:1048800071E0FDD3648094804031900C73E0547FDC
:10489000F0ED75F00312013C900C74F0D3940340DA
:1048A000037403F0900C71E0FF900C74E075F0035A
:1048B000A4FEC3EF9E900C71F0803B900C73E0441B
:1048C00080F0900C71E0FF3395E0FEC374029FFF0F
:1048D000E49EFE7C007D031201BD900C74EFF0D3CA
:1048E000940340037403F0900C74E075F003A4FF8C
:1048F000900C71E02FF0900C72E0FF900C74E0C40B
:10490000333354C0FEEF4E900C72F0A3E0FD7F05F0
:1049100012757A900C72E0FD7F0A12757A900C7114
:10492000E0FF22E4900C65F0900E1EE0900C64F025
:1049300012376B900C65EFF0E060030249E01268FB
:10494000B8900B16E07002A3E07009900C65740932
:10495000F00249E0900E21E0700CA3E07008A3E0A3
:104960007004A3E06024900C697401F0A3740EF04D
:10497000A37421F0900B4BE0FBA3E0FAA3E0F91243
:104980003A84900C65EFF0E07056900E25E0900CA4
:1049900062F0FE900E20E0FF900C6A7401F0A374A8
:1049A0000EF0A37426F0A3EEF0900E1FE0900C6EB4
:1049B000F0A37401F0A3740CF0A37465F0900B4B9A
:1049C000E0FBA3E0FAA3E0F9125468900C63EFF067
:1049D000900C62E06F6009900C65E0700374FFF06A
:1049E000E4FF127462900D6C7436F0A37404F090BE
:1049F0000C65E0900D6EF0900C63E0900D6FF09000
:104A00000E73E0FBA3E0FAA3E02401F9E43AFA1202
:104A1000015E900E72F0A37401F0A3740DF0A37404
:104A20006CF0027520900C63EBF0A3EAF0A3E9F0C0
:104A30002425F9E43AFA900C827401F0A3740CF086
:104A4000A37469F0125167EF6008E4900B59F0A36A
:104A5000F022784D768F087691E47821F6087680FA
:104A60000876E0087602900C66E0FBA3E0FAA3E08B
:104A7000F912015EFF900C69E0FE6F08F6E924016F
:104A8000F9E43AFA12015EFF900C6AE0FD6F08F655
:104A9000900C66E0FBA3E0FAA3E02402F9E43AFA02
:104AA00012015EFFEE6F08F6900C66E0FBA3E0FAE1
:104AB000A3E02403F9E43AFA12015EFFED6F08F671
:104AC000900C63E0FBA3E0FAA3E02425F9E43AFAB2
:104AD00012015E08F6900C63E0FBA3E0FAA3E02469
:104AE00026F9E43AFA12015E08F67D367F0D12755A
:104AF0007A7F8F1276B0E4900B59F0A3F0900C8A75
:104B0000741DF0A3E4F0A37400F0A37421F0A37467
:104B10000AF07B007A00794E7D01126CC4900C6320
:104B2000125BE922900C86EBF0A3EAF0A3E9F0AC6B
:104B3000071255DB900C95EFF0E4900C8AF0EF3300
:104B400095E0FEEF25E0FFEE33FE74822FF9740E40
:104B50003EFA7B01E4FD122D9E900C95E02FF09023
:104B60000C89E0900C8BF0FD900C95122D87900C29
:104B700095E02FF0AF04900C8CEFF0FD900C9512A7
:104B80002D87900C95E02FF0A37403F0900C96E025
:104B9000FFC36480948B505B900C86E0FBA3E475AC
:104BA000F001120209A9F0FA12015EFEEFFD339541
:104BB000E0FC748A2DF582740C3CF583EEF0900CC9
:104BC00095E0FF3395E0FEEF25E0FFEE33FE7482C3
:104BD0002FF9740E3EFA7B01748A2DF582740C3C19
:104BE000F583E0FD122D9E900C95E02FF0A3E004DC
:104BF000F080997B017A0C798A7D0B7C001260250C
:104C0000AD07AC06900C95126DE0900C95E02FF07E
:104C10007B017A0E7982E0FD3395E0FC02754B90C2
:104C20000C91EBF0A3EAF0A3E9F0A3EDF0E4FFA30D
:104C3000E0FBA3E0FAA3E0F912015EFE900C91E024
:104C4000FBA3E0FAA3E02402F9E43AFAEE12019998
:104C5000900C95E0FBA3E0FAA3E02401F9E43AFA12
:104C600012015EFE900C91E0FBA3E0FAA3E02403A6
:104C7000F9E43AFAEE120199900C94E0FEEFC39E2B
:104C80005032900C98E0FBA3E0FAA3E02FF9E43A4D
:104C9000FA12015EFE900C91E0FBA3E0FAA3E0247F
:104CA00004F9E43AFAEF7C0029F9EC3AFAEE120141
:104CB000990F80C4900C94E0FF900C91E0FBA3E06E
:104CC000FAA3E02424F9E43AFAEF120199900C9B3C
:104CD000E0FBA3E0FAA3E0F912015EFF900C91E083
:104CE000FBA3E0FAA3E02425F9E43AFAEF120199D4
:104CF000900C9BE0FBA3E0FAA3E02401F9E43AFA6C
:104D000012015EFF900C91E0FBA3E0FAA3E02426E1
:104D1000F9E43AFAEF020199900C63EBF0A3EAF0A0
:104D2000A3E9F02425F9E43AFA900C827401F0A387
:104D3000740CF0A37469F0125167EF6008E4900BF3
:104D400059F0A3F022784D768F087691E47821F619
:104D50000876700876E008760708F6900C66E0FBA7
:104D6000A3E0FAA3E0F912015EFF900C69E06F087E
:104D7000F6E92401F9E43AFA12015EFF900C6AE0C8
:104D80006F08F6900C63E0FBA3E0FAA3E02425F99A
:104D9000E43AFA12015E08F6900C63E0FBA3E0FA35
:104DA000A3E02426F9E43AFA12015E08F67D367F84
:104DB0000D12757A7F8F1276B0E4900B59F0A3F044
:104DC000900C8A741DF0A3E4F0A37400F0A3742186
:104DD000F0A37409F07B007A00794E7D01126CC457
:104DE000900C63E0FBA3E0FAA3E02425F9E43AFA8F
:104DF000C002C001A3E0F9A3E0FAA3E0900C6EC9E1
:104E0000F0A3EAF0A3E9F0D001D00212522B22E481
:104E1000900C94F0900C93F0900C93E0FFC39419D5
:104E20005059EF64126013EF6414600EEF64156064
:104E300009EF64166004EFB41722900C94E0FF04AD
:104E4000F0EF75F003A424AEF9740C35F0FA7B0191
:104E5000900C93E0FF7D0312710A8017900C93E091
:104E6000FF1273C9900C93E02495F582E4340CF59D
:104E700083EFF0900C93E004F0809DC2A17F017E4F
:104E8000001276F5D2A17F017E001276F5E4900C37
:104E900094F0900C93F0900C93E0FFC39419505948
:104EA000EF64126013EF6414600EEF64156009EF95
:104EB00064166004EFB41726900C94E0FF04F0EF42
:104EC00075F003A424AEF9740C35F0FA7B01900C54
:104ED00093E0FF900CC17403F0126AE38013900C0E
:104EE00093E0FF2495F582E4340CF583E0FD127520
:104EF0007A900C93E004F0809D22900F6AEFF0A36B
:104F00007403F0A374E8F0900E72E0FFA3E0FBA33B
:104F1000E0FAA3E02401F9E43AFAEF120199900FC4
:104F200022E064017031900F22E0B40117900F6B02
:104F300074FFF5F01201F345F060097F647E001202
:104F4000790780E2900F6BE07002A3E070097BFFAD
:104F50007A7779A312108BE4900F6AF0A2AF9200D7
:104F6000C2AFE59620E7FB75960E759701E5962092
:104F7000E7FB759691E59620E7FBAF97900F22E04F
:104F8000FEB4030DE59620E7FB759611759710802A
:104F900046EE7043900F2204F0EF30E50BE59620CB
:104FA000E7FB759611759740EF30E20BE59620E729
:104FB000FB759611E4F597900E72E0FD7C00A3E07E
:104FC000FBA3E0FAA3E0F97F21126E38E59620E713
:104FD000FB759611759701A20092AF22900C637435
:104FE000FFF0E4900C62F0900C62E0FFFDD3900BB8
:104FF00017E09D900B16E09400405FEF75F028A439
:10500000241AF9740135F0FA7B01781F7C0E7D01BA
:105010007E007F081205BEEF703812376B900C636C
:10502000EFF07029900E27E0FD900C897401F0A339
:10503000740DF0A37470F0900E28E0900C8CF07B4F
:10504000017A0E791F124121900C63EFF0E4FF12F8
:105050007462900C62E004F0808D900D6C7450F0DE
:10506000A37440F0900C63E0FF3395E0FE7CFF7D7D
:10507000FF1201AB900D6EEFF0900E28E0900D6FD7
:10508000F07B017A0D796C900E73EBF0A3EAF0A33C
:10509000E9F02401F9E43AFA12015E900E72F0028E
:1050A0007520900C66EBF0A3EAF0A3E9F0784D765A
:1050B0008F087691E47821F60876590876C5A3E042
:1050C000FBA3E0FAA3E0F912015E08F6E92401F976
:1050D000E43AFA12015E08F6900C66E0FBA3E0FAEF
:1050E000A3E02425F9E43AFA12015EFFC4540FFE4E
:1050F000900C69E0FBA3E0FAA3E02402F9E43AFA99
:1051000012015E54F04E08F6900C66E0FBA3E0FA44
:10511000A3E02426F9E43AFA12015EFEC4540FFD1E
:10512000EFC454F04D08F6EEC454F008F67D367F17
:105130000D12757A7F8F1276B0E4900B59F0A3F0C0
:10514000900C8A741DF0A3E4F0A37400F0A3742102
:10515000F0A37408F07B007A00794E7D01126CC4D4
:10516000900C66125BE922900C857401F0784D7604
:105170008F087690E47821F60876300876C112011F
:105180005E08F6E92401F9E43AFA12015E08F6E451
:10519000900B59F0A3F0FD7F1A12757A7D207F1BCA
:1051A00012757A7F8F1276B0900C8A741DF0A3E48A
:1051B000F0A37400F0A37421F0A37405F07B007ACF
:1051C00000794E7D01126CC47F807E001271927F47
:1051D0008F1276B07F5F7E00127192900B5AE03092
:1051E000E629E0541E6008900C857401F08028E4E4
:1051F000900B59F0A3F0900C82E0FBA3E0FAA3E03F
:10520000F91279ACE4900C85F0800CE4900B59F025
:10521000A3F0900C8504F0E4FD7F1B12757AE490F6
:105220000B59F0A3F0900C85E0FF22900C6BEBF093
:10523000A3EAF0A3E9F0900C717404F07F807E0083
:10524000127192E4900B59F0A3F07F8F1276B07D2B
:105250003F7F0D12757A7D147C007F527E00126DA7
:1052600022900B5AE030E677900C6EE0FBA3E0FA58
:10527000A3E0F97F021279687B017A0C79727F02D0
:105280001279687F8F1276B0900B5AE030E323904A
:105290000C6EE0FBA3E0FAA3E0F912015E44801279
:1052A0000199900C6EE0FBA3E0FAA3E0F912015E15
:1052B0008029900C6BE0FBA3E0FAA3E0F912015EF9
:1052C000FF900C72E06F6012E92401F9E43AFA12DF
:1052D000015EFF900C73E0B50705E4900C71F0E4FB
:1052E000900B59F0A3F0900C71E0FF22900F17E0A3
:1052F0007010A3E0700C900F1BE07006A3E0640236
:105300006003127750900F15E0247F601314603211
:1053100024027072900F19E07017A3E06015806688
:10532000900F11E0B4040A900F19E07004A3E0603C
:10533000028053900F1274FFF0A37481F0A3748A5B
:105340008036900F11E0B40406900F19E0600280DF
:1053500035900F1AE0B4812C900F22E0900F12B418
:10536000030C74FFF0A37481F0A37488800A74FFA7
:10537000F0A37481F0A3748AF0900F1FE4F0A3747B
:1053800002F080058000127750900F21E0640460E5
:1053900018E59620E7FB759611759740900F2174DC
:1053A00001F0E4900F1DF0A3F022900C6374FDF067
:1053B000E4900C62F0900C62E0FFFDD3900B17E0DC
:1053C0009D900B16E09400405FEF75F028A4241A1E
:1053D000F9740135F0FA7B01781F7C0E7D017E00A7
:1053E0007F081205BEEF703812376B900C63EFF038
:1053F0007029900E27E0FD900C687401F0A3740EE4
:10540000F0A37429F0900E28E0900C6BF07B017AE9
:105410000E791F123120900C63EFF0E4FF127462DA
:10542000900C62E004F0808D900D6C7448F0A374D1
:1054300003F0900C63E0FF3395E0FE7CFF7DFF12EC
:1054400001AB900D6EEFF07B017A0D796C900E73CD
:10545000EBF0A3EAF0A3E9F02401F9E43AFA12012F
:105460005E900E72F0027520900C66EFF0A3EBF0E8
:10547000A3EAF0A3E9F0E4900C72F0A3F0900C6DB5
:10548000E0FF900C73E0C39F400302551CE4A3F0BF
:10549000900C73E0FC900C66E02C900C79F0EC75AD
:1054A000F002A4FF900C6AE0FBA3E0FAA3E02FF95E
:1054B000EA35F0FA900C7AEBF0A3EAF0A3E9F09069
:1054C0000C6EE0FD900C67E0FBA3E0FAA3E0F9129C
:1054D00045EB900C72EFF0900C74E004F0E0C39494
:1054E00007500C900C72E060061275F3EF70A190FB
:1054F0000B42E06006900C72740AF0900C72E0FFB0
:105500006011900C6FE0FBA3E0FAA3E0F9EF120149
:10551000998009900C73E004F002547D900C73E0C4
:10552000FF22900C62E4F0A3F0A3F0900B5BE0B4D8
:105530000110900C6274FFF0A37461F0A374E3F0A7
:105540008038900E1FE0146013047020900C627479
:10555000FFF0A37461F0A374F7F0801E900C6274E6
:10556000FFF0A37462F0A3741AF0800E900C6274C2
:10557000FFF0A37462F0A3743CF07F31900D6EE4F1
:10558000F0A3DFFC900D6C7411F0900C62E0FBA3B3
:10559000E0FAA3E0F9127642EF04900D6DF0900C62
:1055A000D37401F0A3740DF0A3746EF0900D6DE050
:1055B00024FE900CD6F0900C62E0FBA3E0FAA3E08E
:1055C000F9127219900E737401F0A3740DF0A374A4
:1055D0006CF0900E727431F00275207B017A0E79B6
:1055E00082900C9BEBF0A3EAF0A3E9F0900C9BE017
:1055F000FBA3E0FAA3E0F97455120199900C9BE02B
:10560000FBA3E0FAA3E02402F9E43AFA745512018C
:1056100099900C9BE0FBA3E0FAA3E02404F9E43AA0
:10562000FA7473120199900C9BE0FBA3E0FAA3E0DB
:105630002406F9E43AFA740A120199900C9BE0FBF3
:10564000A3E0FAA3E02401F9E43AFA7408120199FC
:10565000900C9BE0FBA3E0FAA3E02403F9E43AFA00
:105660007408120199900C9BE0FBA3E0FAA3E024DC
:1056700005F9E43AFA7408120199900C9BE0FBA337
:10568000E0FAA3E02407F9E43AFA7404120199FF5E
:1056900022900C63EBF0A3EAF0A3E9F0784D768F4B
:1056A000087691E47821F60876430876E0087603D8
:1056B000ED60050876808004E47825F6900C63E0C0
:1056C000FBA3E0FAA3E02425F9E43AFA12015EFF15
:1056D00054FEC313782546F6EF5401C433333354D4
:1056E00080FF900C63E0FBA3E0FAA3E02426F9E43A
:1056F0003AFA12015EFE54FEC3134F08F6EE54014F
:10570000C4333333548008F67D367F0D12757A7FAB
:105710008F1276B0E4900B59F0A3F0900C8A741DB0
:10572000F0A3E4F0A37400F0A37421F0A37407F0D5
:105730007B007A00794E7D01126CC4900C63125B81
:10574000E922900F55EBF0A3EAF0A3E9F0900F5592
:10575000E0FBA3E0FAA3E02402F9E43AFA12015EC6
:10576000900CD3F0900F55A3E0FAA3E02403F9E4E2
:105770003AFA12015E900CD4F07BFF7A5D79C51283
:10578000108B7BFF7A5D79D912108BE4900F58F063
:10579000A3F0900F55E0FBA3E0FAA3E02424F9E482
:1057A0003AFA12015EFF900F58E0FCA3E0FDC39FA0
:1057B000EC94005034900F55A3E0FAA3E02404F9D0
:1057C000E43AFAE92DF9EA3CFA12015E900CD3F0C2
:1057D0007BFF7A5D79E412108B900F59E004F07032
:1057E000B1900F58E004F080A97BFF7A5D79EA025E
:1057F000108B900B4EE0B40102E4F0900E1FE060BD
:1058000006A3E0900B43F0900E21E06006A3E09029
:105810000B44F0900E23E06006A3E0900B45F0905F
:105820000E25E06006A3E0900B46F0900E27E060A6
:1058300006A3E0900B4AF0900E29E06006A3E0FF7B
:1058400012481D7E007F407D007B017A0D796C122D
:1058500005E2900D6C745AF0A37440F0900B43E095
:10586000900D6FF0900B44E0900D71F0900B45E0BF
:10587000900D73F0900B46E0900D75F0900B4AE0A0
:10588000900D77F0126B9F900D79EFF0900E72747F
:1058900040F0A37401F0A3740DF0A3746CF00275D2
:1058A00020C0E0C0F0C083C082C0D075D000C0006E
:1058B000C001C002C003C004C005C006C007E59611
:1058C00020E7FB759686E59620E7FB900CCCE597E4
:1058D000F0E59620E7FB759682E59620E7FB900CB5
:1058E000CDE597F0E59620E7FB759684E59620E7F1
:1058F000FB900CCEE597F0900CCCE030E1031278F1
:10590000A3900CCCE030E203127733900CCDE03062
:10591000E0031214C5900CCDE030E10312796F90D2
:105920000CCEE030E10312692A900CCCE030E003A9
:105930001278B2D007D006D005D004D003D002D060
:1059400001D000D0D0D082D083D0F0D0E032C0E0FF
:10595000C0F0C083C082C0D075D000C000C001C0FC
:1059600002C003C004C005C006C007127987900BAF
:1059700058EFF0127987AC07900B55E4F0900B5874
:10598000E0FE4F543F900D19F0EE54C0FF6009E067
:10599000FEECF45FFFEE4FF0900D19E0900B58F025
:1059A00030E523127981900B55EFF0541FC3941208
:1059B0004004E04480F0900B55E0FF541FD3940660
:1059C0005004EF4440F0900B55E0FE900D19E0FDBF
:1059D000EDFF900B59E04EF0A3E04FF0D007D0065A
:1059E000D005D004D003D002D001D000D0D0D082D6
:1059F000D083D0F0D0E032E4900C62F0126B3B1216
:105A0000376B900C62EFF0E4900B16F0A3F0EF70A0
:105A1000377B01900C6C04F0A3740EF0A37420F09B
:105A2000900E1FE0900C6FF0E4A3F0A374FFF0A3BE
:105A30007475F0A374F3F07A0179167D01122316C0
:105A4000900B16EEF0A3EFF0E4FF127462900B16C9
:105A5000E07002A3E0900B4B60127401F0A374019C
:105A6000F0A37416F0E4900C62F0800CE4F0A3F064
:105A7000A3F0900C627409F0900D6C7434F0A37470
:105A800003F0900C62E0900D6EF0900E727403F0D3
:105A9000A37401F0A3740DF0A3746CF00275209050
:105AA0000C63EBF0A3EAF0A3E9F02425F9E43AFA59
:105AB000900C827401F0A3740CF0A37466F0125180
:105AC00067EF6008E4900B59F0A3F022784D768FD1
:105AD000087691E47821F60876400876E0087601A9
:105AE000900C63E0FBA3E0FAA3E02425F9E43AFA82
:105AF00012015E08F6900C63E0FBA3E0FAA3E02439
:105B000026F9E43AFA12015E08F67D367F0D127529
:105B10007A7F8F1276B0E4900B59F0A3F0900C8A44
:105B2000741DF0A3E4F0A37400F0A37421F0A37437
:105B300006F07B007A00794E7D01126CC4900C63F4
:105B4000125BE922900C63EBF0A3EAF0A3E9F024E6
:105B500025F9E43AFA900C827401F0A3740CF0A3D6
:105B60007466F0125167EF6008E4900B59F0A3F0EF
:105B700022784D768F087691E47821F608764008F1
:105B800076E0087605900C63E0FBA3E0FAA3E0243E
:105B900025F9E43AFA12015E08F6900C63E0FBA3E3
:105BA000E0FAA3E02426F9E43AFA12015E08F67D51
:105BB000367F0D12757A7F8F1276B0E4900B59F014
:105BC000A3F0900C8A741DF0A3E4F0A37400F0A37A
:105BD0007421F0A37406F07B007A00794E7D0112E7
:105BE0006CC4900C63125BE922E0FBA3E0FAA3E033
:105BF0002425F9E43AFA900C7FEBF0A3EAF0A3E94C
:105C0000F0A37404F07F807E00127192E4900B592F
:105C1000F0A3F07F8F1276B07D3F7F0D12757A7DF5
:105C2000147C007F527E00126D22900B5AE030E609
:105C30004D7B017A0C79837F021279687F8F12760F
:105C4000B0900B5AE030E309900C83E04480F08080
:105C500029900C7FE0FBA3E0FAA3E0F912015EFFBC
:105C6000900C83E06F6012E92401F9E43AFA120122
:105C70005EFF900C84E0B50705E4900C82F0E490A0
:105C80000B59F0A3F0900C82E0FF227B017A0C7993
:105C90006E7D08900C9BEBF0A3EAF0A3E9F0A3ED76
:105CA000F0E4900CA1F0900B59E0FFA3E0900C9F62
:105CB000CFF0A3EFF0E4900B59F0A3F07D067F0145
:105CC00012757A7D03E4FF12757A900C9FE0FEA3B3
:105CD000E0FF30E106A374FBF08044EF30E408906D
:105CE0000CA174FFF08038EF30E62E7F1C1273C9D0
:105CF000EF541FFE900C9EE0FFB50615900C9BE044
:105D0000FBA3E0FAA3E0F9127968E4900CA1F0801B
:105D10000E900CA174FEF08006900CA174FDF07F33
:105D20008F1276B0900CA1E0FF22E4900F51F0E4C6
:105D3000900F52F0A3F0A3F0900F50F0900C6CE491
:105D4000F0A3F0A3F0A3F0900F51E0900C70F0A33B
:105D500074FFF0A37479F0A374C4F07B017A017925
:105D6000167D10122316EFFD900F54E02DF0900FCA
:105D700053E03400F0900F52E0FEEFD39E4002EF6C
:105D8000F0900F50E004F0E0C394FF40AF7BFF7A47
:105D9000687942900F51E0900CD3F0900F53E0FFE0
:105DA000A3E0900CD4CFF0A3EFF0900F52E0900C52
:105DB000D6F012108B900F51E004F0E0C3940F5016
:105DC00003025D2F225072696E74205043202568B3
:105DD000687820256868780A005072696E742045DA
:105DE000504320002568687820000A00544147206D
:105DF000256868783A0A00524E31363A202568689C
:105E00007820256868780A004E756D626572206F8B
:105E10006620726561642062797465733A20256436
:105E20000A0050433A202568687820256868780081
:105E30004550433A20004550434C454E2028627956
:105E4000746573293A20256868640A0048414E4405
:105E50004C453A202568687820256868780A00ED66
:105E6000603575A5FF900D25E06010C2A8C2A0E4C2
:105E7000F590D2A07590800000C2A0AF051DEF6024
:105E80001612015EF59000D2A0000000C2A07401BD
:105E900029F9E43AFA80E4900D23E06034E4F5A5B2
:105EA0007590FF900D23E0FF14F0EF60247590FFD4
:105EB000D2A000900D20E0FBA3E0FAA3E0F9E5906A
:105EC000120199C2A0900D21E475F0011201F38036
:105ED000D275A5FF900D24E0FFB4020DC2A0E4F539
:105EE00090007590800000F590EFB4010B759080E4
:105EF00000D2A0E4F590C2A022900C62EFF0D394FF
:105F00000F40037489F0900C62E02424F582E4349D
:105F10000FF583E0900C64F0E0C4135407900C6319
:105F2000F0900C63E0FFD39400404DC2A2EF14FF49
:105F300074017E00A807088005C333CE33CED8F99C
:105F4000FF900C64E0FDEF5D7BFF600D7A68796D7A
:105F500012108B7FC27E01800B7A68796F12108BD2
:105F60007F967E001276F5D2A27F967E001276F59D
:105F7000900C63E014F080A97BFF7A687971900C33
:105F800062E0900CD3F012108B7FC27E010276F596
:105F9000900D6C741DF0900E1FE0FF64126013EF03
:105FA0006414600EEF64156009EF64166004EFB4CA
:105FB00017287B017A0C79627D0312710A900CD349
:105FC0007401F0A3740DF0A3746EF0A37403F07B5E
:105FD000017A0C7962127219802E900E1FE0FF1266
:105FE00073C9900C62EFF0900CD37401F0A3740DA0
:105FF000F0A3746EF0A37401F0FB7A0C7962127254
:1060000019E4900D6FF0A3F0900D6C741DF0A37463
:1060100006F0900E72F0A37401F0A3740DF0A37457
:106020006CF0027520900C9BEBF0A3EAF0A3E9F072
:10603000A3ECF0A3EDF074FF900CA2F0A3F0E490B9
:106040000CA0F0A3F0900C9EE0FEA3E0FFC3900C28
:10605000A1E09FEE6480F8900CA0E064809850511D
:10606000900C9BE0FBA3E475F001120209A9F0FA81
:1060700012015EFD900CA2E0FAA3E0FBEAFFEF6DD7
:1060800025E0FFE433FE74882FF582747F3EF583AC
:10609000EBFEE4936EFF740193900CA2CFF0A3EF9C
:1060A000F0900CA1E004F0709C900CA0E004F08053
:1060B00094900CA2E0FEA3E0FF22E4900F5FF0902A
:1060C0000F5FE0FFC3941F400302614E7BFF7A65C0
:1060D00079A6900CD3EFF012108B900F5FE0FF6465
:1060E000126014EF6414600FEF6415600AEF641619
:1060F0006005EF641770387A0F79601271067BFFC4
:106100007A6579B3900F62E0900CD3F012108B7B1C
:10611000FF7A6579B3900F61E0900CD3F012108B89
:106120007BFF7A6579B3900F60E0900CD38012907A
:106130000F5FE0FF1273C97BFF7A6579B9900CD3CA
:10614000EFF012108B900F5FE004F00260BF22901E
:106150000C637402F0900D6C7458F0E4900C62F0D3
:10616000900C62E0FFC3941F505AEF64126013EF6B
:106170006414600EEF64156009EF64166004EFB4F8
:10618000171D900C63E07C00246CF9EC340DFA7B55
:10619000017D0312710A900C63E02403F0801D90CE
:1061A0000C62E0FF1273C9900C63E0246CF582E48A
:1061B000340DF583EFF0900C63E004F0900C62E096
:1061C00004F0809C900C63E02402900D6DF0900E22
:1061D000727440F0A37401F0A3740DF0A3746CF01A
:1061E00002752063617574696F6E2077726F6E67D8
:1061F00020636869700A00415333393932204D6990
:106200006E6920526561646572204669726D7761BE
:10621000726520312E352E310A004153333939321F
:1062200020524F4745522052656164657220486193
:1062300072647761726520312E320A0057726F6E78
:10624000672076657273696F6E207479706520734C
:10625000656E64004B494C4C205461670A006E6FB8
:10626000206E65656420746F2061636365737320BD
:106270005461670A00900F67EBF0A3EAF0A3E9F01E
:106280007430120199900F67E0FBA3E0FAA3E024B9
:1062900001F9E43AFA7478120199EF7804A2E7134D
:1062A000D8FB540FFED394095005EE2430800574BA
:1062B000F62E2441FD900F67E0FBA3E0FAA3E02453
:1062C00002F9E43AFAED120199EF540FFED3940962
:1062D0005005EE2430800574F62E2441FF900F67A0
:1062E000E0FBA3E0FAA3E02403F9E43AFAEF120199
:1062F00099900F67E0FBA3E0FAA3E02404F9E43AE5
:10630000FAE4020199787FE4F6D8FD75815075D9D9
:106310000002634F020BCFE493A3F8E493A340037E
:10632000F68001F208DFF48029E493A3F8540724EF
:106330000CC8C333C4540F4420C8834004F45680AF
:106340000146F6DFE4800B01020408102040809033
:1063500027F1E47E019360BCA3FF543F30E509546C
:106360001FFEE493A360010ECF54C025E060A84057
:10637000B8E493A3FAE493A3F8E493A3C8C582C84E
:10638000CAC583CAF0A3C8C582C8CAC583CADFE923
:10639000DEE780BE7BFF7A62795412108B12376B76
:1063A000900C62EFF0703E1268B8900B16E070022D
:1063B000A3E07008900C627409F08029900C667458
:1063C00001F0A3740EF0A3741FF0900E23E0900C64
:1063D00069F0900B4BE0FBA3E0FAA3E0F91244C78D
:1063E000900C62EFF0E4FF127462900D6C743EF05A
:1063F000A37404F0900C62E0900D6EF0900E73E0C8
:10640000FBA3E0FAA3E02401F9E43AFA12015E905A
:106410000E72F0A37401F0A3740DF0A3746CF0027B
:106420007520900F11E064047061900F15E0FF601B
:106430005A64016056900F17E07050900F19E07089
:106440004A900F1BE07044A3E06002803E900F155D
:10645000E064027036900F18E07030900F1AE0FF81
:1064600064816005EF64027022EFB48121E596201B
:10647000E7FB75960E759701E59620E7FB7596117B
:10648000759710900F227403F08003127750E596F1
:1064900020E7FB75960EE4F597900F21E064046009
:1064A0000BE59620E7FB75961175974822900F1122
:1064B000E064026025900F15E0701F900F19E070E6
:1064C00019A3E07015A3E07011A3E0700D900F17F1
:1064D000E07007A3E0D39401400512775080449008
:1064E0000F18E0D394004031900F117404F0E49041
:1064F0000F22F0E59620E7FB75960E759701E5965D
:1065000020E7FB759612759704E59620E7FB7596D4
:106510000EE4F59712796F800A900F117403F090D2
:106520000F22F0900F21E06404600BE59620E7FB5A
:1065300075961175974822256868782025686878CF
:10654000202568687820256868780A00454E207004
:10655000696E206661696C65640A0043616E6E6FE6
:10656000742072756E206F6E204153333939300AB2
:106570000043616E6E6F742072756E206F6E2041E5
:1065800053333939310A00556E6B6E6F776E206365
:1065900068697020256868780A00494E5456434F50
:1065A0005F6C776D0A000A7265672025686878203D
:1065B0002020002568687820002568687800900F02
:1065C00011E06404705B900F15E0FF60546401609B
:1065D00050900F17E0704A900F19E07044900F1B15
:1065E000E0703EA3E060028038900F15E064027016
:1065F00030900F18E0702A900F1AE0FF648170212C
:10660000EFB48120E59620E7FB75960E759701E5BE
:106610009620E7FB759611759740E4900F22F08065
:1066200003127750E59620E7FB75960EE4F59790F8
:106630000F21E06404600BE59620E7FB7596117569
:10664000974822900E1FE0FF900C62F064126014D5
:10665000E0FE6414600EEE64156009EE64166004DA
:10666000EEB417117B017A0E7920900CC17403F0FF
:10667000126AE3801E900C62E0C39480500D900E6D
:106680001FE0FFA3E0FD12757A8008900C62E0FF26
:106690001276B0900D6C741BF0A37403F0E4A3F0B9
:1066A000900E73E0FBA3E0FAA3E02401F9E43AFAC8
:1066B00012015E900E72F0A37401F0A3740DF0A3AA
:1066C000746CF0027520900F15E06480701C900FC0
:1066D00017E07016A3E07012A3E0700EA3E0700A3A
:1066E000A3E07006A3E06401600512775080389043
:1066F0000F11E0FFB40416900F1274FFF0A3748121
:10670000F0A37488F0900F1FE4F0A304F0EFB4033B
:1067100016900F1274FFF0A37481F0A3748AF090A6
:106720000F1FE4F0A304F0900F21E064046018E56B
:106730009620E7FB759611759740900F217401F034
:10674000E4900F1DF0A3F022C0E0C083C082C0D04F
:1067500075D000C000C001C002C003C006C00778E9
:1067600012E66051C2CF08860308E6FA08E6240163
:10677000F9E43AFA74FF120177FF7813860308E60A
:10678000FA08E6F912015EFEA807088002C313D8D2
:10679000FCFF7813860308E6FA08E62401F9E43AD8
:1067A000FA12015E700B740226F618E436F67812BF
:1067B00016EF139293D007D006D003D002D001D0A9
:1067C00000D0D0D082D083D0E032900F5AEBF0A32B
:1067D000EAF0A3E9F012798D900F5EEFF0900F5D73
:1067E0007433F0C2A8900D20E4F0A3F0A3F0A3F05E
:1067F000A3F0A304F0FB7A0F795DFD125E5F900DAC
:1068000020E4F0A3F0A3F0A3F0A3F0A3F07B017ABF
:106810000F795E7D01125E5F900F5AE0FBA3E0FAF4
:10682000A3E02401F9E43AFA900D20E4F0A3F0A3E8
:10683000F0A3F0A37402F0E4A3F07DFB125E5FD23C
:10684000A822666F756E64207769746820706F7710
:10685000536C6F743D2568687820257820746167D3
:10686000732C206D617820256868780A002D002E31
:106870000020256868780A0048656C6C6F20726F8C
:1068800067657220554846205246494420576F722A
:106890006C640A006C776D5F617333393978496EC7
:1068A000697469616C697A652829207265747572EA
:1068B0006E65642025780A00900B4BA3E0FAA3E0F4
:1068C0004A7003FEFF22900B4BE0FBA3E0FAA3E02B
:1068D0002404F9E43AFA900C6CEBF0A3EAF0A3E993
:1068E000F0900B4BA3E0FAA3E02424F9E43AFA1267
:1068F000015E900C6FF0E4A3F0A374FFF0A3747535
:10690000F0A374F3F07B017A01793E7D0112231626
:10691000900B16EEF0A3EFF04E600E900B4B74014F
:10692000F0A37401F0A3743EF022E4900CCFF0E5E4
:106930009620E7FB75960E759701E59620E7FB75A7
:106940009694E59620E7FBAF97900F22E0B4030CF6
:10695000E59620E7FB75961475972022EF30E60B3D
:10696000E59620E7FB75961475978012002E900E21
:106970005DE0FD7C00A37F21126C64900E5EE0FB65
:10698000A3E0FAA3E0F912015EFF126D80E5962004
:10699000E7FB759614E4F59722900C7DEFF07F8F5E
:1069A0001276B0784D768F087698E47821F6900EBE
:1069B000E9E03333335418FF900EECE0C433542035
:1069C0004FFF900EEBE025E025E054044FF6900CCD
:1069D0007DE025E0541EFF900EEAE0FEC433335400
:1069E000C04F08F6900C8A741FF0A3E4F0A3740063
:1069F000F0A37421F0A37402F07B007A00794E7D3D
:106A000001026CC4900F11E064047024900F15E033
:106A10006481701C900F17E07016A3E07012A3E061
:106A2000700EA3E0700AA3E07006A3E064016005A5
:106A30001277508016900F1274FFF0A37481F0A3A8
:106A4000748AF0900F1FE4F0A304F0900F21E0642B
:106A5000046018E59620E7FB759611759740900F36
:106A6000217401F0E4900F1DF0A3F022900C85EF4B
:106A7000F0D2937F017E001276F51255DB900C86E2
:106A8000EFF03395E0FEEF25E0FFEE33FE74822F4A
:106A9000F9740E3EFA7B01900C85E0FD122D9E905C
:106AA0000C86E02FF07B017A0C79857D017C001249
:106AB0006025AD07AC06900C86126DE0900C86E068
:106AC0002FF07B017A0E7982E0FD3395E0FC1275A0
:106AD0004BD29322F07A0C79767B01900CC174032F
:106AE000F07F14900CBDEFF0A3EBF0A3EAF0A3E964
:106AF000F0900CBDE04420F0C2A8900D20E4F0A37B
:106B0000F0A3F0A3F0A3F0A304F0FB7A0C79BDFD91
:106B1000125E5F900CC1E0FD900D20E4F0A3F0A3A5
:106B2000F0A3F0A37402F0E4A3F0900CBEE0FBA38A
:106B3000E0FAA3E0F9125E5FD2A822900C6874011B
:106B4000F0A37401F0A37416F0E4FFFEFD8046E4A8
:106B5000FF7E0AFDFC900C64E0F8A3E0F9A3E0FAE4
:106B6000A3E0FBC312039C5035900C68E0FBA3E448
:106B700075F001120209A9F0FAE4120199900C646F
:106B8000E0FCA3E0FDA3E0FEA3E02401FFE43EFE61
:106B9000E43DFDE43CFC900C641203D380B122E49C
:106BA000900C62F07F051273C9900C631273C5EFED
:106BB00030E211900C62E024B5F0EF30E020E024E8
:106BC00005F0801A900C62E024B9F0EF30E004E0A8
:106BD0002408F0EF30E107900C62E024F6F0EFC4F7
:106BE0001313540375F003A4FF900C63E0900C6240
:106BF00030E706E0C39FF08003E02FF0900C62E0E6
:106C0000FF22900C7DEBF0A3EAF0A3E9F0E4A3F0FF
:106C1000A3F07FC0FE1271927F5F7E00127192908E
:106C20000B5AE020E022E0541E6008900C8174FFB3
:106C3000F08026900C7DE0FBA3E0FAA3E0F9121AA5
:106C4000E7900C81EFF08011900C7DE0FBA3E0FA5F
:106C5000A3E0F9E4F5F012024A7F8F1276B0900CAF
:106C600081E0FF22E0FBA3E0FAA3E0F9900CD0EF73
:106C7000F0900CD3EBF0A3EAF0A3E9F0900CD1EC88
:106C8000F0A3EDF04C603C900CD0E0F5964396C03C
:106C9000E4FFFED3900CD2E09F900CD1E09E402008
:106CA000E59620E7FB900CD3E0FBA3E0FAA3E02FEE
:106CB000F9EA3EFAE5971201990FBF00010E80D361
:106CC000E4F59622900C8AE04420F0C2A8900D20B2
:106CD000E4F0A3F0A3F0A3F0A3F0A304F0125E5F2E
:106CE000900D20E4F0A3F0A3F0A3F0A3F0A3F07BB9
:106CF000017A0C798A7D01125E5F900C8EE0FD9026
:106D00000D20E4F0A3F0A3F0A3F0A37402F0E4A339
:106D1000F0900C8BE0FBA3E0FAA3E0F9125E5FD2E7
:106D2000A822900C85EEF0A3EFF0A3ECF0A3EDF019
:106D3000900C85E0FEA3E0FF900B59E05EFEA3E01F
:106D40005F4E7026900C87E07002A3E0601CE59116
:106D500030E7DD7FE87E03127667900C88E024FF41
:106D6000F0900C87E034FFF080C6900C87E0700252
:106D7000A3E0700B124E0F900B59E4F0A304F02225
:106D8000900E71E0703204F0900CD3F0A3740EF00A
:106D9000A3741DF0900E5EE0FBA3E0FAA3E02401D3
:106DA000F9E43AFA12015E04900CD6F0900E5EA35C
:106DB000E0FAA3E0F9027219900E5EE0FBA3E0FA9C
:106DC000A3E0F912015E900CD3F0900E1DE0900C40
:106DD000D4F07BFF7A7579CA12108B22AD07AC060E
:106DE000E0FF3395E0FEEF25E0FFEE33FE74822FE7
:106DF000F9740E3EFA7B01900C9BEBF0A3EAF0A332
:106E0000E9F0A3ECF0A3EDF0F4FFECF4FE900C9E9F
:106E1000F0A3EFF0EEFD122D9E900C9CE475F004B3
:106E20001201F3900C9BE0FBA3E0FAA3E0F9A3A30B
:106E3000E0FD122D9E7F0422900F44EFF0900F474B
:106E4000EBF0A3EAF0A3E9F0900F45ECF0A3EDF02E
:106E50004C603BE59620E7FB900F44E0F596E4FF9D
:106E6000FED3900F46E09F900F45E09E4020900F8C
:106E700047E0FBA3E0FAA3E02FF9EA3EFA12015E35
:106E8000F597E59620E7FB0FBF00010E80D3229017
:106E90000CD0EFF0900CD3EBF0A3EAF0A3E9F09064
:106EA0000CD1ECF0A3EDF04C603BE59620E7FB90B5
:106EB0000CD0E0F596E4FFFED3900CD2E09F900C4E
:106EC000D1E09E4020900CD3E0FBA3E0FAA3E02F9A
:106ED000F9EA3EFA12015EF597E59620E7FB0FBF4F
:106EE00000010E80D322C0E0C083C082C0D075D024
:106EF00000C000C001C002C003C299790CE7780B42
:106F00006670057811F68018780D860308E6FA0891
:106F1000E6F9780CE60629F9E43AFA12015EF599E9
:106F2000309806780A7601C298D003D002D001D0FA
:106F300000D0D0D082D083D0E032900F15E0701D09
:106F4000900F19E07017A3E07013A3E0700FA3E097
:106F5000700B900F17E07005A3E030E70312775035
:106F6000900F217405F0900F18E0900F11600574D8
:106F700003F080037402F0900F21E06404600BE5DD
:106F80009620E7FB75961175974822740B2FF582B2
:106F9000740D3EF583E0FF900DB8E0600BE4F090D7
:106FA0000DB7F07811E670FB900DB7E024B9F582CB
:106FB000E4340DF583EFF0900DB7E004F0E0FDC38D
:106FC00094645004EFB40A0F7B017A0D79B91274FE
:106FD00095900DB87401F022900CD0EFF0E4A3F07E
:106FE000900CD1E0FFD394035039EF25E025E02445
:106FF00076F582E4340EF583E0FF900CD0E0FEEFEE
:10700000B50618A3E025E025E02477F582E4340EE8
:10701000F583A3E0FAA3E0F9020405900CD1E004A3
:10702000F080BD22E59620E7FB759601759708E58F
:107030009620E7FB759607759707E59620E7FB75A1
:107040009609759707E59620E7FB75960B759707E8
:1070500075D7E0E59620E7FB75960F75978043E6B8
:1070600002D2AFE59620E7FB759601759701229055
:107070000F18E0FF126FD8900E73E0F9A3E0FAA3A7
:10708000E0900F12C9F0A3EAF0A3E9F0900E72E0CD
:10709000FF900F1FE4F0A3EFF0900F21E064046075
:1070A00018E59620E7FB759611759740900F2174AF
:1070B00001F0E4900F1DF0A3F02212002E900E5E5E
:1070C000E0F9A3E0FAA3E0900F12C9F0A3EAF0A35D
:1070D000E9F0900F1BE0FFA3E0900F1FCFF0A3EFAC
:1070E000F0900F21E064046018E59620E7FB7596A8
:1070F00011759740900F217402F0E4900F1DF0A3DA
:10710000F0227A0C79767B017D03900CBDEFF0A321
:10711000EBF0A3EAF0A3E9F0C2A8900CBDE0446054
:10712000F0A3E0F9A3E0FAA3E0900D20C9F0A3EAF0
:10713000F0A3E9F0A3EDF0A37402F0A314F0FB7A3E
:107140000C79BDFD125E5FD2A8227F0A1273C9902E
:107150000C9BEFF07D227F0112757A900C9BE0FD75
:107160007F0A12757AE4FF1273FB7F8F1276B07D6F
:10717000507F1B12757A7F971276B07D43E4FF1221
:1071800076D3C292D2937F017E001276F5C2A80216
:1071900079C0900C91EEF0A3EFF0E4FFFE900C911B
:1071A000E0FCA3E0FD900B59E05CFCA3E05D4C70BB
:1071B00010C3EF94FDEE94FF50070FBF00010E8047
:1071C000DCD3EF94F0EE94FF400B124E0F900B596E
:1071D000E4F0A304F022900E1FE004600E14701778
:1071E000D28243C701C2B0E4FF8009C28253C7FE06
:1071F000D2B07F01127462900D6C7419F0A3740305
:10720000F0E4A3F0900E727403F0A37401F0A37481
:107210000DF0A3746CF0027520900CD0EBF0A3EA93
:10722000F0A3E9F0E4FF900CD6E0FEEFC39E5029F6
:10723000900CD0E0FBA3E0FAA3E02FF9E43AFA12B5
:10724000015EFE900CD3E0FBA3E0FAA3E02FF9E48B
:107250003AFAEE1201990F80CD22900C64EFF09073
:107260000B4EE0FE6F6031EE24FE600804700812E1
:1072700079E980031279DF900C64E024FE600E044B
:10728000700E7B017A0B79431279E28003127959EF
:10729000900C64E0900B4EF022D2937F067E001299
:1072A00076F5900C7C74AAF0900C7EF0900C8074B3
:1072B0000AF0900C7D7408F0900C7FF0900C8174B3
:1072C00004F07B017A0C797C7D037C0012754BD233
:1072D000937F017E000276F5E4780AF67811F6785D
:1072E0000BF608F6900DB8F0900DB7F0C29FD29D46
:1072F000D29C758840758920438E08758D30D28E5A
:1073000043A41075E10175B283D2BC75A890D2ACCC
:10731000D2AF43E24022900F15E06401701C900F41
:107320001BE07016A3E07012900F17E0700CA3E042
:107330007008A3E07004A3E06003127750900F215F
:10734000E06404600BE59620E7FB7596117597489D
:107350002274FF900C62F0A3F0EE3395E0FDFCE4A4
:107360007B30FAF9F8120269C374FF9F900C63F046
:1073700074FF9E900C62F0E4F5C8438E30E0FEA3EB
:10738000E0FDF5CA8DCCEEF5CBF5CD22900E1EE0DA
:10739000B40431900D6C7456F0A37403F07B017A41
:1073A0000D796C900E73EBF0A3EAF0A3E9F02401E1
:1073B000F9E43AFA12015E900E72F0900D6E74FFCD
:1073C000F012752022EFF07F0A900D1AEFF0C2A89C
:1073D000E04440F0900D207401F0A3740DF0A3740C
:1073E0001BF0A37401F0A3F0A3F0FB7A0D791AFD52
:1073F000125E5FD2A8900D1BE0FF22900C9CEFF074
:1074000070077D407F0912757A900C9CE0B40607E6
:107410007D807F0912757A7F031273C9EF540FFFC5
:10742000900C9CE0FEC454F04FFD7F0302757A126D
:107430007975EF602C900E1DE075F003A424EAF539
:1074400082E5F03479F583E4740193FA740293F9D8
:10745000120405900B47E0700312797BE4900B4710
:10746000F022900C71EFF0E4FF1273C9900C71E000
:107470006008EF4401FFC2828006EF54FEFFD28213
:10748000AD07E4FF12757A900C71E060077F027E11
:10749000001276F522E4900D18F07811E670FB7872
:1074A000117601780DA60308A60208A601780C76CD
:1074B00001AF0518A607780D860308E6FA08E6F975
:1074C00012015EF59922A2AF9201C2AF75FF8075DD
:1074D000EF028E088F0975B7A575B7F1438F017557
:1074E000FF8075EF02850982850883EDF0538FFEDA
:1074F000A20192AF22900D6C7405F0900D6AE0909D
:107500000D6DF0900D6BE0900D6EF0900E737401A8
:10751000F0A3740DF0A3746CF0900E727403F0225B
:10752000E4900C71F0900D6DE0FF900C71E0FEC3E3
:107530009F5017746C2EF582E4340DF583E0FF1232
:1075400078DD900C71E004F080DB227813A603084C
:10755000A60208A601E408F6AF057812A60775C8CA
:1075600004AFA875A820D2AF7812E670FB30CFFD2B
:107570008FA8E4F5C8227D02E4FF900CBDEFF0A3D4
:10758000EDF0C2A8900D20E4F0A3F0A3F0A3F0A3C7
:1075900004F0A3F0FB7A0C79BD7D02125E5FD2A8E5
:1075A00022900F64EBF0A3EAF0A3E9F0900F64E0FF
:1075B000FBA3E0FAA3E0F9127800AD07900F64E0B6
:1075C000FBA3E0FAA3E0F90274957573622065727B
:1075D000726F72202D207265706F7274202568683A
:1075E00078206C6F737420616674657220256868FA
:1075F000780A00900B3FE07002A3E070037F012245
:1076000012783DC3900B40E09F900B3FE09E5009E5
:10761000900B427401F07F00227F01227F96127648
:10762000B07F971276B07FF47E011279077F0F1238
:1076300073C9900C81EFF07F961276B0900C81E0C8
:10764000FF22900C65EBF0A3EAF0A3E9F0E4FF90D1
:107650000C65E0FBA3E0FAA3E02FF9E43AFA12018B
:107660005E60030F80E9227C007D0412040BC3746A
:10767000FF9FFF74FF9EFC538EBFE4F591EFFBF577
:1076800092ECF5938B94F59543910422438E045329
:1076900088EF53D8BFE58954F04401F589E4F58AB1
:1076A000F58C75D90475D840F5F9F5FA43881022A0
:1076B000900CA2EFF0C2A8900D20E4F0A3F0A3F08C
:1076C000A3F0A304F0A3F0FB7A0C79A2FD125E5F95
:1076D000D2A822900C9CEFF0A3EDF0900D20E4F0E6
:1076E000A3F0A3F0A3F0A3F0A304F0FB7A0C799C21
:1076F0007D02025E5F900CBDEEF0A3EFF0900CBD3A
:1077000074FFF5F012020945F060097FE87E03126C
:10771000790780E92243B203E4F5B943B9801278CE
:107720009443B9C0127894E5B930E5FB75B690750D
:10773000A90322900F117402F0E59620E7FB7596DD
:1077400001759701E4900F21F0A37403F0A3F022D8
:10775000E59620E7FB75960EE4F597E59620E7FBA6
:10776000759611759720900F217404F0227F397E51
:1077700000E4FDFCC3ED9FEE6480F8EC648098505B
:10778000070DBD00010C80EC2275F003EFA424EA84
:10779000F582E5F03479F583740193FA740293F974
:1077A0000204050A0A53656E645061636B657420B8
:1077B00074696D6564206F75740A0A00900E5EE04E
:1077C000FBA3E0FAA3E02401F9E43AFA12015E9087
:1077D0000DB5F022123D53127520900E1F7402F069
:1077E000900D6EE06003B401EB221229E2127520C5
:1077F000900E1F7402F0900D6EE06003B401EB2256
:10780000E4FFFE12015E600C0FEF70010E09E970DB
:10781000F20A80EF22900F21E06404600BE59620CD
:10782000E7FB75961175974822900B56E0FD7F0592
:1078300012757A900B57E0FD7F0A02757AAFFA7ED7
:1078400000ADF97C00ABFAEBB507F2EFFEEDFF22DD
:1078500075A5FF7590800000D2A000E4F59000C2ED
:10786000A022E4900B59F0A3F0C292D29312785068
:10787000D2A8227F051273C9900B561273C5900BC4
:1078800057EFF022E4900C62F0A3F0900B4EF090D2
:107890000B47F022E4FFFE0FBF00010EBE01F8BF50
:1078A000F4F522900CD0E004F07006900CCFE004C8
:1078B000F022900CD0E004F07006900CCFE004F0C1
:1078C00022D287D28375E40BD288D2A8D2AF2212FB
:1078D00079101278C1E4F590C2A0D2A1227811E605
:1078E00070FB781176018F9922780AE670FBE478B4
:1078F0000AF622E4900C62F0A3F00277157F0D7E69
:10790000001273517F0022127667E59130E7FB2267
:10791000C2A143A60743E240227F0212725A024FDD
:10792000DC7F0212725A0253AA7F0112725A025964
:10793000F77F0112725A0249237F0112725A0243E1
:10794000937F0112725A023BFA7F0112725A02634C
:10795000947F0112725A023E97E4FF1273FB7F007C
:1079600022E4780AF6AF9922AD077F1F02710AE47C
:10797000900F22F022900E71E0FF22E4900E71F041
:10798000227F1C1273C9227F0C1273C9227F13122B
:1079900073C922E4780AF6227F15026A6C7F0A0214
:1079A0006A6C7F09026A6C7F08026A6C7F02027946
:1079B000687F9D0276B07F9E0276B07F800276B0AF
:1079C00075A59F227F01220279E80255220271D615
:1079D000026643025F9002614F0257F27F00227FEE
:1079E00000220232B92222222222FF79C7FF79C760
:1079F000FF79C7FF79C7FF79C7FF79C7FF79C7FF4D
:107A000079C7FF79C7FF79C7FF79C7FF79C7FF79C2
:107A1000C7FF79C7FF79C7FF79C7FF79CAFF79C761
:107A2000FF79C7FF79C7FF79C7FF79C7FF79C7FF1C
:107A300079C7FF79CDFF79C7FF79D0FF79C7FF7983
:107A4000D3FF79C7FF79C7FF79C7FF79C7FF79C728
:107A5000FF79C7FF79C7FF79C7FF79C7FF79C7FFEC
:107A600079C7FF79C7FF79C7FF79C7FF79C7FF7962
:107A7000C7FF79C7FF79C7FF79C7FF79C7FF77D4F9
:107A8000FF79C7FF7929FF79C7FF7931FF79C7FFF0
:107A90007939FF79C7FF79C7FF79C7FF7941FF7946
:107AA000C7FF7949FF79C7FF425AFF79C7FF0663CD
:107AB000FF79C7FF77EAFF79C7FF7951FF79C7FFE1
:107AC0007921FF79C7FF7919FF79C7FF79C7FF7956
:107AD000C7FF79C7FF79C7FF79C7FF79C7FF79C7A4
:107AE000FF79C7FF79C7FF79C7FF738CFF79C7FF9D
:107AF00079D6FF79C7FF79D9FF79C7FF79C7FF79B1
:107B0000C7FF79C7FF79C7FF79C7FF79C7FF79C773
:107B1000FF79C7FF79C7FF79C7FF79C7FF79C7FF2B
:107B200079C7FF79C7FF79C7FF79C7FF79C7FF79A1
:107B3000C7FF79C7FF79C7FF79C7FF79C7FF79C743
:107B4000FF79C7FF79C7FF79C7FF79C7FF79C7FFFB
:107B500079C7FF79C7FF79C7FF79C7FF79C7FF7971
:107B6000C7FF79C7FF79C7FF79C7FF79C7FF79C713
:107B7000FF79C7FF79C7FF79C7FF79C7FF79C7FFCB
:107B800079C7FF79C7FF79C7FF79C7FF79C7FF7941
:107B9000C7FF79C7FF79C7FF79C7FF79C7FF79C7E3
:107BA000FF79C7FF79C7FF79C7FF79C7FF79C7FF9B
:107BB00079C7FF79C7FF79C7FF79C7FF79C7FF7911
:107BC000C7FF79C7FF79C7FF79C7FF79C7FF79C7B3
:107BD000FF79C7FF79C7FF79C7FF79C7FF79C7FF6B
:107BE00079C7FF79C7FF79C7FF79C7FF79C7FF79E1
:107BF000C7FF79C7FF79C7FF79C7FF79C7FF79C783
:107C0000FF79C7FF79C7FF79C7FF79C7FF79C7FF3A
:107C100079C7FF79C7FF79C7FF79C7FF79C7FF79B0
:107C2000C7FF79C7FF79C7FF79C7FF79C7FF79C752
:107C3000FF79C7FF79C7FF79C7FF79C7FF79C7FF0A
:107C400079C7FF79C7FF79C7FF79C7FF79C7FF7980
:107C5000C7FF79C7FF79C7FF79C7FF79C7FF79C722
:107C6000FF79C7FF79C7FF79C7FF79C7FF79C7FFDA
:107C700079C7FF79C7FF79C7FF79C7FF79C7FF7950
:107C8000C7FF79C7FF79C7FF79C7FF79C7FF79C7F2
:107C9000FF79C7FF79C7FF79C7FF79C7FF79C7FFAA
:107CA00079C7FF79C7FF79C7FF79C7FF79C7FF7920
:107CB000C7FF79C7FF79C7FF79C7FF79C7FF79C7C2
:107CC000FF79C7FF79C7FF79C7FF79C7FF79C7FF7A
:107CD00079C7FF79C7FF79C7FF79C7FF79C7FF79F0
:107CE000C7FF79C7FF79C7FF79C7120110010000EC
:107CF0000040251329C000000102000109022900EB
:107D000001010080AF090400000203000000092106
:107D1000010100012242020705810340000A070514
:107D2000020340000A0600FF0901A1018510950227
:107D3000750826FF0015000901910285119530751F
:107D40000826FF001500090181028531950275089A
:107D500026FF001500090191028532953F7508261E
:107D6000FF001500090181028533953F750826FF44
:107D70000015000901910285349502750826FF005F
:107D800015000901810285189502750826FF001566
:107D9000000901910285199502750826FF0015005A
:107DA000090181028535953F750826FF00150009F8
:107DB00001910285369503750826FF00150009011B
:107DC000810285379507750826FF00150009019186
:107DD000028538953F750826FF00150009018102CC
:107DE000851C9502750826FF001500090191028582
:107DF0001D9505750826FF00150009018102851AE9
:107E00009505750826FF00150009019102851B954F
:107E100002750826FF00150009018102853F950CB7
:107E2000750826FF001500090191028540950C7523
:107E30000826FF001500090181028547953F750856
:107E400026FF001500090191028548950275082654
:107E5000FF001500090181028549950C750826FF70
:107E6000001500090191028550953F750826FF0015
:107E70001500090181028541953F750826FF00150F
:107E800000090191028542953F750826FF00150003
:107E90000901810285439502750826FF0015000936
:107EA0000191028544953F750826FF0015000901E0
:107EB0008102853B9507750826FF00150009019191
:107EC00002853E9502750826FF0015000901810212
:107ED000853D9506750826FF00150009019102856C
:107EE0003C9502750826FF001500090181028545B1
:107EF0009509750826FF0015000901910285469530
:107F000004750826FF001500090181028555953F7B
:107F1000750826FF00150009019102855695027526
:107F20000826FF001500090181028558953F750854
:107F300026FF001500090181028557950175082665
:107F4000FF00150009019102855A953F750826FF2B
:107F5000001500090181028559953F750826FF002B
:107F6000150009019102C005030904000A0341003C
:107F70004D005300200000000E0341005300330069
:107F80003900390031000000000010212042306328
:107F9000408450A560C670E781089129A14AB16B61
:107FA000C18CD1ADE1CEF1EF123102103273225209
:107FB00052B5429472F762D693398318B37BA35AB1
:107FC000D3BDC39CF3FFE3DE2462344304201401D9
:107FD00064E674C744A45485A56AB54B8528950901
:107FE000E5EEF5CFC5ACD58D3653267216110630A9
:107FF00076D766F6569546B4B75BA77A9719873851
:10800000F7DFE7FED79DC7BC48C458E5688678A768
:108010000840186128023823C9CCD9EDE98EF9AFA0
:1080200089489969A90AB92B5AF54AD47AB76A9648
:108030001A710A503A332A12DBFDCBDCFBBFEB9EF0
:108040009B798B58BB3BAB1A6CA67C874CE45CC518
:108050002C223C030C601C41EDAEFD8FCDECDDCD40
:10806000AD2ABD0B8D689D497E976EB65ED54EF4E8
:108070003E132E321E510E70FF9FEFBEDFDDCFFC90
:10808000BF1BAF3A9F598F78918881A9B1CAA1EBE4
:10809000D10CC12DF14EE16F108000A130C220E360
:1080A000500440257046606783B99398A3FBB3DA08
:1080B000C33DD31CE37FF35E02B1129022F332D2B0
:1080C0004235521462777256B5EAA5CB95A88589D8
:1080D000F56EE54FD52CC50D34E224C314A0048100
:1080E0007466644754244405A7DBB7FA879997B8A8
:1080F000E75FF77EC71DD73C26D336F2069116B050
:108100006657767646155634D94CC96DF90EE92F67
:1081100099C889E9B98AA9AB58444865780668279F
:1081200018C008E1388228A3CB7DDB5CEB3FFB1E47
:108130008BF99BD8ABBBBB9A4A755A546A377A16EF
:108140000AF11AD02AB33A92FD2EED0FDD6CCD4D17
:10815000BDAAAD8B9DE88DC97C266C075C644C453F
:108160003CA22C831CE00CC1EF1FFF3ECF5DDF7CE7
:10817000AF9BBFBA8FD99FF86E177E364E555E748F
:0C8180002E933EB20ED11EF00100000054
:00000001FF
